:10000000F01F0010014D0000FF4C0000FF4C0000ED
:10001000FF4C0000FF4C0000FF4C000000000000FF
:10002000000000000000000000000000FF4C000085
:10003000FF4C000000000000FF4C0000E921000020
:10004000F11F0000F11F0000F11F0000F11F000070
:10005000F11F0000F11F0000F11F0000F11F000060
:10006000F11F0000F11F0000F11F0000F11F000050
:10007000F11F0000FD4C0000FD4C0000C10000001D
:10008000B1220000C9220000DD240000F524000098
:10009000FD4C000039260000FD4C0000FD4C000026
:1000A000FD4C0000FD4C0000FD4C0000FD4C00002C
:1000B000FD4C0000FD4C0000FD4C0000FD4C00001C
:1000C000554B10B51A6801321A60544B1A68544BDC
:1000D000D2B2302A69D01ADC182A44D012DC082A9D
:1000E00032D0102A00D094E04E4A002111604E49CF
:1000F0000A68501C08604D49895C4D4AC9B21160BC
:10010000282287E0202A63D0282A32D081E0482A9A
:100110005ED004DC382A51D0402A53D079E0502AEE
:1001200060D0582A75D13F490A68501C0860404980
:1001300008684049C0B288543F4A0221FF3111602B
:1001400080221021D20563E0374A00211160116836
:10015000481C1060354A515C354AC9B211602822EA
:100160001A6001223CE030490A68501C08602F499F
:1001700009E02D4A314910680968884207D21168A0
:10018000481C1060294A515C294AC9B240E02C4AF7
:1001900011688022D205002901D0202138E02649AB
:1001A0000220FF300860102132E08022D2051021A9
:1001B000116008221A608122520011E08221490058
:1001C0001D4A25E01E4A1168042201291AD11DE0AA
:1001D0008022D2051021116008221A600422FF3209
:1001E000154B17E00F4A1168481C1060104804684E
:1001F0001048E4B244541068114A116804220139CD
:10020000884203D28021C9050A6002E01A6000E03A
:10021000116008221A6010BD900300100400004015
:1002200018000040840300108C030010A405001087
:10023000080000409405001088030010B405001069
:10024000900500101B4B02211A6810B50A431A6072
:10025000194B20211A68041C0A431A60174B1849CD
:100260001A680A401A601868012210431860154B7A
:1002700018680140196019680A431A60124B6C2211
:100280001A60124B1249186804F0C0FD114A106040
:10029000114A1060022C02D1104BA0221A60104BA0
:1002A000802212021A6080234022DB0501201A609E
:1002B00010BDC046048004408080044030400440AB
:1002C000F8FCFFFF3440044018000040880500108F
:1002D000400D030014000040100000400C000040DE
:1002E00000E100E0034B1B689A06FBD5024B186047
:1002F0007047C0461480004000800040FFFFFFFFB1
:1003000070B5061C00200D1C01F066F9002801D014
:1003100002F068FD00242C60301C3460291C01F0C0
:1003200089F9201C01F058F9A04207D002F05AFDCB
:100330002C60301C3460291C01F07CF970BD08B5BC
:1003400001F082FF08BD08B500230B60036001F0D7
:1003500071F908BD10B502F00DFD0D4B00201968B4
:1003600002F032F9002002F01FF9002002F0FCF840
:10037000084B01241C60084B201C198801F0E0FF89
:10038000201C01F0CDFF201C01F0AAFF10BDC046CB
:1003900084050010800300108C05001008B50A20A9
:1003A000002101F01DFFFFF7D5FF08BD08B50020B3
:1003B00002F0EAF8012001F0A3FF02F0E1FC08BD21
:1003C00038B5051C0C1CFFF7C5FF054B0122281C86
:1003D000211C5A6203F0BAFFFFF7E8FF38BDC046A0
:1003E000600D001010B5041CFFF7B4FF201C03F0D3
:1003F00035FF041CFFF7DAFF201C10BD08B50020F4
:10040000FFF7F0FF08BD000008B5021C02490348D1
:1004100002F038FB08BDC0463C4F0000344F0000DE
:1004200037B500F04FFF0322164B1748002101F0AB
:1004300037F800F051FFFFF7E1FF1448FFF7E4FF42
:10044000134B144A00241A601D1C2B689C4211DABD
:1004500002F0D4F9002803D001F0A6FC00240FE03C
:100460000A2001F0F1FE684601A9FFF749FF009B51
:10047000002B05D0FFF7C2FF074802F003FB37BD92
:100480000134E2E708000010454F0000544F00001F
:1004900074040010701700005A4F000070470000ED
:1004A0001B4B73B5041C1B49186804F0AFFC1A49B8
:1004B00000901A4A1A4B201C02F0F0FA01F096F94B
:1004C000002812D001F0AEF9FA218900061C04F0D0
:1004D0009DFC051C201C02F032FB124B20186B43C4
:1004E0001149F3182A1C02F0D9FA201C02F027FB4C
:1004F0000E4B20181B68002B02D003DA0C4A02E0D6
:100500000C4A00E00C4A0D4902F0C8FA73BDC0461F
:100510008805001040420F006B4F00003C4F000068
:10052000784F000018FCFFFF7C4F000050020010C5
:10053000684F0000654F000018970000874F0000CB
:1005400070B5051C0E1C141C00F0BCFE301C291CD0
:100550000022064B00F0A4FF201C01210922044BBD
:1005600000F09EFF00F0B8FE70BDC046080000100D
:100570001400001000B5084B89B01A78074B684684
:100580001B78074902F08AFA01206946054AFFF7FD
:10059000D7FF09B000BDC046440200101000001093
:1005A000BB4F0000C94F0000F0B52A4C2A4D2378FC
:1005B00085B001932F78FFF7DDFFFFF71FFF0026BF
:1005C00002A803A9FFF79CFE029800282BD0C0B216
:1005D00000F080FF40280CD004D830280ED03928F5
:1005E00017D01BE0462830D049280DD0412815D11E
:1005F00026E02B783E2B11D8013303E02B78002B1B
:100600000CD0013B2B7009E02378062B06D8013370
:1006100003E02378002B01D0013B237000F03EFE65
:10062000FFF7A8FF0026029B002B02D0C82001F094
:100630000BFE04200321013601F0D2FD1D2EBFDD8B
:10064000019B2F70237000F029FEFFF7D7FE05B045
:10065000F0BDC046100000104402001038B5051C63
:100660000C1C00F0FAFD291C221C0120FFF768FF7A
:10067000034B00225A60034A943212689A6038BDD4
:10068000600D0010C405001010B590B0041C684641
:10069000FFF706FF201C69466A46FFF751FF10B0BE
:1006A00010BD000000B52D228DB0002800D02B22F7
:1006B00068460D4902F0F2F904A802F025FC012079
:1006C000694604AAFFF73CFF0320002101F088FDE2
:1006D0000220FFF787FE0028EED00A20002101F05B
:1006E0007FFD0DB000BDC046DD4F000070B58CB081
:1006F000FFF784FE02A8144902F02AFA2E25FF35DE
:1007000004AE301C02F000FC6846002409A9093040
:10071000F47402F01DFA02AA0420311CFFF710FF46
:10072000201C032101F05CFD684601A9019400949E
:10073000FFF7E6FD009BA34202D1013DA542DFD1B8
:10074000FFF75CFE0CB070BD19970000F0B50024F7
:1007500093B00594FFF752FE022296230194039270
:10076000251C5B00029300F0ADFD019B9A4F002B0E
:100770006DD10AAE301C02F0C7FB019AF2743274DC
:100780007273B272F2713271002C01D1012D05D158
:10079000301C042100223B1C00F082FE8F4E3B1CCB
:1007A000301C1E21002200F07BFE8B4F012C01D15A
:1007B000012D06D168462D30252100223B1C00F07A
:1007C0006FFE301C332100223B1C00F069FE824E7C
:1007D000022C09D1012D07D0684633304D2100226B
:1007E000331C00F05DFE09E00CA83A210022331C06
:1007F00000F056FE032CEFD1012DEDD0784F331CC5
:10080000381C5921002200F04BFE734E042C01D1FC
:10081000012D06D1684636305F210022331C00F0DE
:100820003FFE381C6C210022331C00F039FE052CE1
:1008300001D1012D06D16846393072210022664B64
:1008400000F02EFE0FA804210922664B03E0664843
:10085000042100223B1C00F023FE00F03DFD059B1F
:10086000002B0AD0143B012B05D8052C03D0962071
:1008700001F0EAFC01E0FFF7C1FD0320011C01F0DB
:10088000AFFC5A4B1E68002EF7D1301C00F0A4FEBE
:1008900006A9071C05A806960596FFF731FD059BDE
:1008A000002B73D007AE08AF301C391C09AA02F028
:1008B0005FFB019000286FD1301C02F043FC051C47
:1008C00005981238052866D804F03EFA0565240C10
:1008D0006503601C00E0601D062104F0EDFA0025B0
:1008E0000C1C59E0052C56D8201C04F02DFA0306E8
:1008F0000B0D10393388013316E0B0780C2104F069
:100900007BFA18E001355DE0387801301AE078783C
:1009100001301FE0052C3ED8201C04F015FA030717
:100920000F1119213388013B338044E0B0780C214A
:100930000A3004F0C1FA0131B1703CE0013D41E000
:1009400038781730182104F0B7FA042239703FE0E4
:1009500078783B303C2104F0AFFA032379702FE024
:100960000023BB70281C072104F0A6FA301C0A1CC7
:100970000991391C052C02D102F055FB02E0039BC2
:1009800002F010FB01259623AB4007E0002F06D1B3
:1009900001235D4003E0012596235B000293059B44
:1009A000842B17D0182B15D0029B029A013B002AEA
:1009B00000D0D7E60EE0301C02F0C4FB0523051C76
:1009C0000393CFE7281C311C02F0ECFB0224052224
:1009D0000392C7E713B0F0BD08000010E64F000017
:1009E000E84F000014000010EA4F000068030010F8
:1009F000F7B502F01FFA18200021FFF7E1FC0024F0
:100A00006B4EFFF7D3FC6B4D00236B62201C02F092
:100A100032FA002C02D00020012101E0062003213F
:100A200001F0DEFB201C02F021FA01A9071C684638
:100A3000002F03D0FFF787FC012728E0FFF783FC96
:100A4000009A002A23D1002CE0D15B4F3B1C983345
:100A50001B68002B0DD1594BF618D7D51820002153
:100A60009437FFF7ADFC3C6863425C4100F0DEFB6D
:100A7000CCE7534B00941A6811321A60009A102A7E
:100A8000E9DC03F09BFB009B01330093F6E7002CAD
:100A90000CD0009B182B01D0002FB2D000F024FC0A
:100AA0004848FFF7B1FC444B0122DA6600F0CCFE67
:100AB00002F02AF9009A182A62D1019F0024F8B2A4
:100AC00000F008FD012601946E62172846D00CD86C
:100AD00013282BD002D8112819D04EE015282DD07C
:100AE00016284AD1FFF760FD4AE026282ED004D808
:100AF00019281ED0212811D03FE0442836D045289F
:100B00003BD1E120000102F0A7FA301C32E02E4B6D
:100B10001B68002B34D0FFF7E9FD05E02A4B1B686A
:100B2000002B2DD0FFF712FE009429E0FFF778FC90
:100B300026E0264B1868301A00F0ACFF0120FFF7C2
:100B4000A3FDFFF75BFCFFF729FC19E0204B052212
:100B50001C70204B1A7000F0A1FB11E01E4B1A68AC
:100B600001321A60032A0BD11C6009E01B4802F015
:100B700073FA201CFFF796FD02E0002301976B62D9
:100B8000FFF7E8FB0098019903F0E0FB6B6A002B8C
:100B900001D0FFF733FC084B94331B68002B03D1C3
:100BA00000F044FB01242BE704F048F827E7C04697
:100BB00020BF0200600D0010C40500100CFEFFFFF6
:100BC00094030010F84F00005002001020000010A5
:100BD00044020010100000101C020010F0F1FFFF92
:100BE00073B501F0F3FF3A4C00F0B8FC394800212E
:100BF00001F072F90021384801F06EF900F086FD2D
:100C000000F026FF23680726B343236023680125ED
:100C10002B4300202360021C0B2101F0E7F8201C6D
:100C20002E4C102101F058F923680022B3432360B1
:100C30002368281C2360042101F0D8F8201C00211F
:100C400001F04AF901F0BCF89620000201F032FDF3
:100C5000234D01235B4200202B60FFF715FD00238D
:100C60002B6050240120FFF7EDFA00F0F1FE02F0B6
:100C7000ABF82B68002B05D16420043C01F0E4FAAA
:100C8000142CEFD10020FFF7FFFC164801F0FAFE0C
:100C9000192001F0D9FA01F0B1FD002802D0FFF7C8
:100CA000BFFB02E0013C002CF2DC02F0E9FA03F0A9
:100CB000A5F91E2300930F2301930B480B490C4AFF
:100CC0000C4B03F0ADF90C4803F0DCF9FFF790FE94
:100CD00074400440984004409C40044094400440C8
:100CE0005002001002500000B94C00000103000047
:100CF0005D0600009403001080030010F7B5002883
:100D00003BD00378303B5A425341C0180378782BCC
:100D100003D101301026012501E00A2600250378C1
:100D2000002201922D2B02D10123013001930023D7
:100D30000278002A1BD0171C303FFCB2092C02D8C5
:100D40007343DB1911E020273A43002D08D0171C0C
:100D5000613FFFB2052F03D81B01573A134304E04C
:100D6000064801F08FFE002007E00130E0E7019A1D
:100D7000002A00D05B420B600120FEBD0C50000039
:100D80000378202B01D10130FAE77047031C303B78
:100D9000DAB2092A01D8181C0AE020231843031CE0
:100DA000613BDBB2052B01D8573801E001204042FE
:100DB000704770B50E1CFFF7E3FF0025041C207878
:100DC000002807D0FFF7E2FF002803DB2D010543D1
:100DD0000134F4E73560201C70BD000008B500F058
:100DE00021FD011C014801F04DFE08BD1A50000014
:100DF00000B589B0684602F087F86946024801F0FC
:100E000041FE09B000BDC04656500000F7B50F1CAA
:100E100001A9161CFFF772FF002814D0019C0B4992
:100E2000201C04F049F80D1C081C642104F044F84F
:100E3000281C3970642103F0E9FF04493070201C3C
:100E400003F0E4FF01E001204042FEBD1027000056
:100E500037B50D1C48686A46694607310632FFF708
:100E6000D5FF01AC69466A4620800132A86802318C
:100E7000FFF7CCFF6B4618702288044B9A4203D9C7
:100E8000201C694602F0CFF837BDC0466B07000052
:100E900007B5486801A9FFF731FF019B3C20584383
:100EA00002F0DAF807BD000007235843054A10187E
:100EB0009C30013B04D3C25C002AFAD0002000E041
:100EC00001207047C405001030B5194885B001F005
:100ED000D9FD0024651CA30719D1201CFFF7E4FFEE
:100EE000002810D0281CFFF7DFFF00280BD0A01C23
:100EF000FFF7DAFF002806D0E01CFFF7D5FF002837
:100F000001D004340EE00B48211C01F0BBFD211C74
:100F1000684602F0C9F9684601F072FE064801F021
:100F2000B1FD2C1CFF2CD5DD01F078FE05B030BDE5
:100F30003C4F0000265000001897000070B50E1CB2
:100F4000FFF71EFF0D25041C0134631E1878FFF700
:100F50001DFF002806DB7055013DF5D2201CFFF770
:100F60000FFF00E0002070BD70B5434C86B02368D1
:100F70000868251C002B06D1404801F083FD03F0D2
:100F80003DF8012309E0012B0DD13D49082201F074
:100F9000E8FD002803D123680133236069E0394864
:100FA00001F070FD5DE00378412B17D1364C023023
:100FB000211CFFF7C3FF002853D00378422B50D1E8
:100FC000211C02300E31FFF7B9FF002849D0037809
:100FD000432B46D1211C02301C3103E0532B06D198
:100FE0002A490230FFF7AAFF002842D139E04D2BF1
:100FF0001FD1274C0230211CFFF7A0FF002830D062
:1010000003784E2B2DD1211C02300E31FFF796FFB5
:10101000002826D00378472B23D1023001A9FFF7FF
:10102000C8FE019B002B1CDB174A1A4853651A495E
:101030001BE001A9FFF7BDFE04782023061C9C439A
:101040000FD1301C02A9FFF779FF019B061CE118A4
:1010500002A802F03FF9002E03D00134042CF0D195
:1010600007E002F0CBFF0B480C4901F00BFD002319
:101070002B6006B070BDC046540300102F50000016
:101080003C4F000045500000C40500100A06001047
:10109000EE05001051500000994F00005B50000019
:1010A00037B54C682378002B25D0201CFFF768FE4D
:1010B00001A9FFF77EFE019B041C002B1BD0D8B2B8
:1010C000FF2B09DD00F022FA019B051C1812C0B2AB
:1010D00000F01CFA019003E000F018FA00250190DE
:1010E0000198002802D0291CFFF76AF923785A1EBC
:1010F0009341E418D6E737BD064A08B513780121B5
:101100004B40137001D0044900E00449044801F049
:10111000B9FC08BD78040010FF4F000062500000C9
:101120006650000007B5486801A9FFF7E7FD019B7D
:10113000002B01DC01230193019B1E2B01DD1E23EB
:1011400001930199034A044B4A4304481A6001F091
:1011500099FC07BD70170000740400107550000062
:1011600038B5051C002D09D0642402200021013C63
:1011700000F062FE002CF8D1013DF3E738BD70B5F8
:10118000061C01200821021C00F080FE072401201B
:101190000821002200F07AFE321C012522412A405B
:1011A0000020022100F072FE281C08212A1C00F0F9
:1011B0006DFE013CEBD270BD10B50021041C0A1C71
:1011C000022000F063FE201CFFF7D9FF10BDF0B530
:1011D000012385B002930023061C039372B60024FA
:1011E00002AB1B59502040421843C0B2FFF7E4FF46
:1011F0000020FFF7E1FF1020FFF7DEFFE020FFF700
:10120000DBFF212767430025F71902200021012277
:1012100000F03CFE785D0135FFF7B1FF842DF4D17D
:101220000434082CDCD162B605B0F0BD08B5AC20A2
:10123000FFF7C2FFAE20FFF7BFFFA520FFF7BCFFFF
:1012400008BD38B50122051C0C1C00F0CFFD281C80
:10125000211C012200F01AFE38BD08B5AF20FFF7AF
:10126000ABFFA420FFF7A8FF08BD08B5AE20FFF72D
:10127000A3FF08BD10B5041CF820FFF79DFF201C3C
:10128000FFF79AFF10BD10B5041C8120FFF794FFF3
:101290003F202040FFF790FF10BD000008B5074B2E
:1012A00020201B781843FFF787FF0A20FFF758FF1D
:1012B000034B1878FFF7E7FF08BDC0461000001089
:1012C0004402001008B5842202480021520001F0B7
:1012D00013FC08BD7904001008B50248FFF777FF3A
:1012E00008BDC0467904001008B501200821FFF7A9
:1012F000A8FF00200221FFF7A4FF02200021FFF732
:10130000A0FF02200621FFF79CFF0320011CFFF72E
:1013100098FF0320011C002200F0B8FD02200621E6
:10132000002200F0B3FD06210122022000F0AEFDF4
:10133000FFF7C8FFFFF7D0FFA220FFF73DFFA02077
:10134000FFF73AFFC020FFF737FF0020FFF792FFBB
:101350000A20FFF705FF4020FFF72EFF2C20FFF7A4
:101360002BFF3220FFF7FCFE2E20FFF725FF322057
:10137000FFF7F6FE2F20FFF71FFF0A20FFF7F0FE12
:10138000FFF78CFFFFF769FF08BD000083280ED828
:101390000F290CD8CB08842253430722C0181140D0
:1013A000034B80220A41111C1A5C114319547047E7
:1013B00079040010F7B55B18DBB20193019B9942E9
:1013C00015D28425CC086C4307270F4080250419CB
:1013D0003D41EFB2A618B44206DA054D65192B78E7
:1013E00001343B432B70F6E70131C9B2E6E7F7BDA4
:1013F00079040010F0B51E1C87B00592F2780491B4
:101400005B68824201D2307845E0244AB478934246
:1014100005D10322041B54430192E4180CE0001B85
:101420000022824204DA1978013202315B18F8E7AF
:101430001A789C1C5B780193A218002503922F1C3C
:10144000019B9F4226DA08220023029200937378C0
:10145000009A9A421CDA029A082A06D1039B9C42FF
:1014600018D00022257802920134EB0708D5049A9F
:10147000009BB818059AC0B29918C9B2FFF786FF49
:10148000009B029A013301326D1000930292DEE755
:101490000137D5E7019807B0F0BDC046995000006C
:1014A000F7B5041C0D1C161C1F1C01F048FB20186E
:1014B0000190019B9C420BD0832D09D82078291CD8
:1014C000321C3B1CFFF796FF01302D180134F0E76A
:1014D000F7BD000010B50021012204230A4C0C5D69
:1014E000844203D118010243D0B20BE0013B002B30
:1014F00004D10132092A00DD1A1C042301312829F4
:10150000ECD1002010BDC046465800000F23020950
:1015100018408000031F00D52833511E00200329E6
:1015200006D8242B04DC04218A1A0249CB18985CC3
:101530007047C0464658000038B5051C0024054BCE
:10154000291CE05C044B0134C01800F0C5FC0A2CD7
:10155000F5D138BD8258000000400440F8B50D4F69
:101560003C68002C15D11020FFF7E6FF0A4B002243
:10157000E65C1B195D78301C291C00F037FC023436
:10158000301C291C012200F081FC142CEED1012317
:101590003B60F8BD480200106E58000070B5002492
:1015A0000B4B0122E65C1B195D78301C291C00F0F6
:1015B0001DFC0234301C291C002200F067FC142C96
:1015C000EED10020FFF7B8FF024B00221A6070BD79
:1015D0006E5800004802001038B5051CFFF7BEFF2A
:1015E000002D09D007210122022000F0FFFB104B43
:1015F00080211A688A431A6000200B2100F01CFC2D
:101600000124002805D000200B2100F015FC4442E5
:101610004441002D09D007210022022000F0E6FB02
:10162000034B80211A680A431A60201C38BDC0464B
:10163000FC3F0250F0B587B00026029001200391D4
:1016400004960596FFF7C8FFB04202D01823049312
:1016500001260021284C009120786178012200F0B9
:10166000C5FB20786178002200F010FC234B9D1D03
:10167000012E24DC6A782F78111C381C019200F0AE
:10168000DBFB002808D100991D4AB3008A5C1033A7
:1016900069465A5001360BE02878697800F0CCFB97
:1016A0000028F0D0381C019900F0C6FB0028EAD0D1
:1016B000009A144B0132023D00929D42D8D1277806
:1016C0006578381C291C002200F090FB291C381C6E
:1016D000012200F0DBFB0C4902348C42BCD100201B
:1016E000864206D0049A029B05991A60039A01204B
:1016F000116007B0F0BDC0466E5800003E580000B3
:10170000465800003C5800008258000008B50120EF
:10171000021C0B2100F06AFB01200B21002200F0CB
:10172000B5FB03200221012200F060FB032002210F
:10173000002200F0ABFB08BD234B37B51A6810211F
:101740008A431A60214B8022196892010A431A6069
:10175000051C0B210120002200F048FB01200B2179
:10176000002200F093FB1A4B9F211A68194C8A4300
:101770001A601A6818491A60184B186803F046FB7B
:101780008023000218432A1C20600221032000F05D
:101790007DFB142000F058FD2368FF229343236053
:1017A00023680F4A134323600E4B1B680193019B70
:1017B000002BF9DA22680C4B13402360FFF7A6FFD9
:1017C00001980004800D3EBD3882044080800440B2
:1017D0009840044000C0014000093D008805001009
:1017E000800000012CC00140FFFFFFF810B50C4C39
:1017F0002068002813DA00202060FFF79DFF0A28E8
:101800000ADC0120FFF798FF0138C023FF385B0096
:10181000984201D801232360FFF778FF206810BDAC
:101820001C00001008B5FFF7E1FF002801D10020DF
:1018300007E00120FFF780FF011EF8D0014803F008
:10184000E5FA08BD50BB120008B5FFF7CFFF00282E
:101850000AD0FFF7E7FFFA22031C0021C00FD200D5
:101860009A424841014B186008BDC0464C02001026
:1018700008B5074B02221A60064BA2221960064BDC
:101880001A70A32258709A7000F0EEFD08BDC04691
:10189000B405001090050010A405001008B5064B13
:1018A00002311960054B00221A60054BA2221A7002
:1018B000587000F0D9FD08BDB40500109005001067
:1018C000A405001070B5051C0E1C0324281C311C37
:1018D000FFF7CEFF0223FF33984202D0013C002CD9
:1018E000F4D170BD70B5051C0E1C0324281C311CDE
:1018F000FFF7D4FF0223FF33984202D0013C002CB3
:10190000F4D170BD0B4B10B51C6800239C420ED067
:10191000094CA31CA270140A5C70140C120EDA702D
:101920009C70FFF7DFFF831EFF3B5A425341181C98
:1019300010BDC04650020010A405001070B50E4C3A
:1019400025680024A54215D00C4C160AA270E6703A
:10195000160C120E6271A371A21D26711C0A54701E
:101960001C0C1B0E9470D370FFF7BCFF841EFF3C51
:1019700063425C41201C70BD50020010A4050010A1
:1019800008B5064B1A6800239A4205D0FFF79AFF64
:10199000831EFF3B5A425341181C08BD50020010E1
:1019A00008B5074B00201B68834207D0022007219F
:1019B000FFF788FF0238FF384342584108BDC04650
:1019C0005002001038B50F4B051C1B6800208342E5
:1019D00017D00924641B631E062B10D8072C05D0D2
:1019E0000948A91E0918221C01F064F8E8B2211C5C
:1019F000FFF778FF0238FF384342584101E00120E9
:101A0000404238BD50020010A6050010012010B55C
:101A1000011CFFF757FF0223FF3398420ED1094BF9
:101A200001211960084B1C78230709D0074B0322BA
:101A300022409A70081CFFF755FF01E00124644220
:101A4000201C10BD5002001094050010A4050010C9
:101A500008B5FFF7DBFF02200121FFF733FF022368
:101A6000FF3398420FD1084B1B787F2B06D9842275
:101A7000022007215204054BFFF760FF09200421D3
:101A8000034AFFF73FFF08BD940500100201140050
:101A90008080808010B500280CD0254B80211A68EA
:101AA0008A431A60234B1B68D907FBD5224B0322BC
:101AB0001A6001E0204B1860204B012200211A60BF
:101AC00019601A60196801221142FBD01C4B802159
:101AD0001A601C4A49021468214311601A1C00282C
:101AE00004D1134B8024196821431960164B1968DF
:101AF00088421CD01860002801D0144800E0144827
:101B0000116803F035F9134BFA2118608900041CA1
:101B100003F07CF91E2358430F4BC821186049017C
:101B2000201C03F073F90D4B186001F039F810BD5B
:101B3000388204400C80044070800440748004406B
:101B4000788004408080044020000010006CDC029B
:101B5000001BB70088050010840500108C050010DC
:101B600008B500F035F9134B00211A68120B120367
:101B70001A60114B1A68120B12031A600F4B1A6885
:101B8000120B12031A600E4B1A68120B12031A6022
:101B90000C4B012219600C4B1A6019601A601A680C
:101BA00001200242FBD0094B23221A60FFF772FF8B
:101BB00008BDC046008000500080015000800250E7
:101BC000008003504080044044800440088004406A
:101BD00038B50F490F4800F055FF0F4D0024281C61
:101BE00000F050FF0D4A0E48A1581219D2682B1C64
:101BF000143400F047FFC82CF4D10A4800F042FF2B
:101C000000F042FB011C084800F03CFF38BDC04614
:101C10003C4F00008C580000DC58000024000010ED
:101C20009E580000A9580000CB580000F0B53B4B6F
:101C30008BB01E68041C002E01D1351C08E0384B07
:101C400002901B6801209B6854E033681E79019D57
:101C50002378002B31D0082D33D02378202B01D1CD
:101C60000134FAE7002B28D06A1CAD0008356B461A
:101C70000192EC50FF2E4CD02278002A07D0631C32
:101C8000202A01D01C1CF7E7002222701C1C019A9C
:101C9000012ADCD1224E234B0B253360371C013D3A
:101CA000002D2ED03B680298196800F06BFF0028C9
:101CB000CBD03B6814333B60F1E7002D1CD0022DE4
:101CC00002D0B54206D911E00398174900F05AFF37
:101CD0000028F6D1124C15482368D96800F0D2FECE
:101CE00023681348196900F0CDFE05E00C4BE8B2FB
:101CF0001B689B6802A99847084A1368002B0BD100
:101D000003E0281C291CFFF763FF0A4800F0BAFE15
:101D100002E0019D0026D2E70BB0F0BD5403001095
:101D20005C03001024000010694F0000D858000028
:101D300056500000DF58000038B5041C164D0A2824
:101D400008D002D8082811D01CE00D2802D07F2826
:101D50000CD017E02A6800231370104800F092FEA0
:101D60000F4C201CFFF762FF2C6013E00C4B2A681D
:101D70009A420FD90B48211C00F084FE2B68013BCE
:101D80002B6007E00748211C00F07CFE2B685A1CE2
:101D90002A601C7038BDC04658030010DC58000093
:101DA00054020010EB58000008B500F027FD002891
:101DB00004D000F0F9FCFFF7BFFFF6E708BD000014
:101DC000014A024B1A607047540200105803001079
:101DD000044B40211A680A431A60034B01221A700F
:101DE0007047C04680800440600300100F4B70B500
:101DF0001B78061C0C1C151C002B01D1FFF7E8FFFB
:101E0000701E022803D80A4B8000C35800E0094B1B
:101E10001A68012D04D1A5402C1C14431C6003E05A
:101E20000121A1408A431A6070BDC04660030010C2
:101E3000D45900000080005038B50F4B051C1B78AA
:101E40000C1C002B01D1FFF7C3FF0020032D12D87B
:101E5000281C012202F078FF02040608074B04E068
:101E6000074B02E0074B00E0074B1B68A240134002
:101E7000181C421E904138BD60030010FC3F00500A
:101E8000FC3F0150FC3F0250FC3F03500F4B70B52C
:101E90001B78061C0C1C151C002B01D1FFF798FFAA
:101EA000701E022803D80A4B8000C35800E0094B7B
:101EB0001A68012D04D1A5402C1C14431C6003E0BA
:101EC0000121A1408A431A6070BDC0466003001022
:101ED000E0590000FC3F005038B5084B041C1B784B
:101EE0000D1C002B01D1FFF773FF236818229343C9
:101EF000236023681D43256038BDC0466003001081
:101F0000054B3F221A60054B01221A60044B402109
:101F10001A688A431A60704724800440D8800440BD
:101F20003882044008B5044B40211A688A431A607D
:101F3000FFF7E6FF08BDC0463882044008B500F050
:101F400059FAFFF72BFB0A480021FFF7C5FF0948A4
:101F50000021FFF7C1FF08480021FFF7BDFF074838
:101F60000021FFF7B9FF06480021FFF7B5FF08BDC4
:101F70000840044000400440AC4004401440044089
:101F80001C40044008B50120FEF75CF908BD0000C4
:101F900008B5114B8022DA675200DA678022D2003E
:101FA000DA6780225201DA6780221201DA67802222
:101FB0009200DA67094A002313600121084A494266
:101FC0001160084A1360084A1360084B01221A6026
:101FD000FFF7D8FF08BDC04604E100E004820440DA
:101FE0000882044004C000403CC0004000C00040E3
:101FF00008B5064B1A6801321A60054B1868FFF7DE
:1020000049FDFFF7C5FFC046C04608BD6403001088
:1020100020000010F7B5071C0C1C72B6FFF78EFFEE
:10202000524B1A68524B1A60002F01D0514B00E0FE
:10203000514B524A04211360514B524D1A680A43C6
:102040001A6000232B60A1071ED04F4B4F4A19681E
:102050000A401A6029684E4BA2070ED5EC225201A5
:102060000A432A6080221A6052001A608022D2003D
:102070001A60802252011A6003E0802212010A4392
:102080002A60802212011A60002F53D0414B002495
:102090001C60414B414E1C60414B301C1C60414B4D
:1020A000211C1C60FFF718FF201C0921221CFFF7D0
:1020B0009DFE201C0921221CFFF7E8FE3A4B8021DF
:1020C0001A683A480A431A60336807229343336018
:1020D00033680222134333600A21784302F048FE3A
:1020E000334B03221860334B1C60334B1A60334B65
:1020F000334A19680A401A601A6880210A431A6034
:10210000234A8B001360204A1168194311602A6822
:10211000022113432B602B4B01221A602A4B1960BA
:102120002A4B1C491A601C601A6018680122104270
:10213000FBD00A60264B012252421A60254B002236
:102140001B680193244B1A6062B630BFC046214B16
:10215000019A1B689A4208D11F4B01221A601F4B3B
:102160001868FFF797FCFFF713FFF7BD38820440AC
:1021700034820440BF180000FF1800003082044081
:1021800010ED00E004820440008204407FE2FFFF83
:1021900000E100E004C0004004000140644004404D
:1021A000044001400480014080800440841E0000FF
:1021B00018C0004008C0004014C000403CC00040AF
:1021C0000FF0FFFF7880044070800440748004406A
:1021D000088204406403001068030010200000100F
:1021E00008B5FFF717FF08BD074B1A68013203D186
:1021F000064A1168013111601A6801321A60044BF5
:102200001A6801321A6070477803001074030010D6
:102210006C030010074B98420AD8074A002313604A
:10222000064A01381060064A1360064B07221A60FE
:102230007047C046FFFFFF007803001014E000E085
:1022400018E000E010E000E00B4A10B51368002829
:1022500000D10120C1438B4208D91168994209D3AA
:10226000591C146809188C42FAD3F6E71168C91A88
:102270008142FBD310BDC04678030010014B1868A3
:102280007047C04678030010064BFA211868064BC9
:1022900010B589001C6802F06BFD044B5C432018EC
:1022A00010BDC04678030010740300103789410048
:1022B000034B01221A60034B1A6801321A607047FF
:1022C00000C000407C030010034B01221A60034B46
:1022D0001A6801321A607047000001408003001044
:1022E000002803D1044B01221A6003E0012801D128
:1022F000024B18607047C04604C000400400014013
:10230000002802D1044B186004E0012802D1034BDD
:1023100000221A607047C04604C00040040001401B
:10232000002801D1044B02E0012804D1034B1A68B4
:1023300002210A431A60704704C0004004000140B3
:1023400010B5002900D1134900280DD1124B80246B
:102350001A6822431A60114B03221860104B19604F
:10236000104B1A60620211E0012811D10A4B802241
:102370001868520002431A600B4B00221A600B4B84
:10238000032219600A4B1A6080229202094B1A60DC
:1023900010BDC046FFFF0000808004407C03001099
:1023A00018C0004014C00040800300101800014015
:1023B0001400014000E100E080231022DB051A60D8
:1023C000094B08221A6000238022D2051268D10628
:1023D00004D5064A934201D00133F5E704489842F8
:1023E0009B4158427047C04618000040FF0F000054
:1023F000FE0F000008B58022154B1202DA67154B5C
:102400006C221A60144B154A19680020114019609B
:1024100019681960124B19680A401A601A68042179
:102420001A600122FFF7E2FC002004210122FFF7DD
:102430002DFD002005210122FFF7D8FC01220020FC
:102440000521FFF723FD074B00221A6008BDC04697
:1024500004E100E01800004030400440F8FCFFFFB9
:102460003440044004800440F8B5174A174C002358
:1024700023601360164A202113608022D205116068
:102480002168144A012903D0934203D00133F7E7AE
:10249000934203D1FFF790FF002014E00E4F002578
:1024A0003E68013E2368FF2B0CD83B689E4204D057
:1024B0003E68FFF7E3FE051C0A35FFF7DFFE8542A5
:1024C000F0D1E7E72068F8BD84030010880300100E
:1024D0008C030010FF0F000090030010034B01223B
:1024E0001A60034B1A6801321A60704700400140BD
:1024F00094030010174B70B501241C60164B1A682A
:1025000012191A60154B1A68002A22D01A68144D45
:10251000013A1A601E68002E0DD02A68201C211C6A
:10252000FFF7B4FC2B68201CE31A2B602A680221F9
:10253000FFF7ACFC0DE01B68201C2B602A68211CF7
:10254000FFF7A4FC2A68201C0221FFF79FFC054B23
:102550001E6070BD008001409C03001098030010B5
:10256000A003001004800140002803D1044B012285
:102570001A6003E0012801D1024B18607047C04681
:102580000440014004800140002802D1044B18603F
:1025900004E0012802D1034B00221A607047C046B4
:1025A0000440014004800140002801D1044B02E0B6
:1025B000012804D1034B1A6802210A431A607047AC
:1025C000044001400480014010B500280FD1124B97
:1025D00080221C68920022431A60104B032218606C
:1025E0000F4B19600F4B1A608022D20211E00128B4
:1025F00011D1094B80221868D20002431A600A4B9D
:1026000000221A60094B03221960094B1A608022CC
:102610001203084B1A6010BD808004409403001020
:1026200018400140144001409C03001018800140F4
:102630001480014000E100E008B5184B1A680E2331
:102640001340062B0DD1164B9E221B68134205D05A
:10265000144ADBB25360144B1B681EE0D9071CD52B
:1026600001E0042B05D1104B1868C0B200F0B1F89E
:1026700013E00C2B06D10B4B8022596852000A4301
:102680005A600AE0022B08D1054B1A68054B9106E7
:1026900001D5002200E001229A6008BD08800040B8
:1026A00014800040A40300100080004000487047E0
:1026B000A4030010F7B52D4B2D4C8022002192036E
:1026C0000191061CDA67201C902200F015FA019B8C
:1026D0000725A360274B284F1A68AA431A60196878
:1026E000012211431960254B1968A9431960196823
:1026F00011431960224B8021186849010143196078
:10270000204B1A6083223A601F4A126819681F4BD7
:102710001868504302F02CFB311C000902F028FB22
:102720001B4B10221B491A60030A0B601A4BC0B2E4
:10273000032218603A60194A1560194A1D1C106876
:102740000190106860230340602BFAD110680123C8
:10275000184202D02B680193F8E723708022114BB6
:1027600092031A6005230B60F7BDC04604E100E048
:10277000A4030010A44004400C800040A840044082
:1027800080800440988004407880044088050010D0
:102790002880004004800040008000400880004005
:1027A0001480004000E100E008B5FFF77FFFC26839
:1027B000031C1202120E8218D07BDA681202120E6B
:1027C0000132D2B29A7352B2002A01DA00229A730D
:1027D00008BD10B5041CFFF769FFC2681204120E91
:1027E0008218D473C2681204120E0132D2B242733C
:1027F00052B2002A01DA0022427310BD08B5FFF779
:1028000055FFC268C36812021B041B0E120ED01AB9
:10281000431E9841C0B208BD70B500241D5D061965
:10282000002D02D005550134F8E7121B301C131C93
:10283000002B03DD0170013B0130F9E7D043C017E5
:102840000240A01870BDF7B5051C01910093561EFB
:10285000092B01D8041C0CE000980A2102F088FA28
:102860000199031C321C281CFFF7EDFF071C2C18D4
:1028700007E0671B002E04DD019B013E237001343D
:10288000F7E700980A2102F0B7FA3031781C21707E
:10289000FEBDF8B50C1CD9175F18051C4F40561E1D
:1028A000092F12D9381C0A21002B03DA02F060FA32
:1028B000434202E002F05CFA031C281C211C321C7B
:1028C000FFF7E7FF041C2D1814E0002B00DA961E1A
:1028D0002A1CA919891A002902DD14700132F8E7AF
:1028E000F443E41734402D19002B03DA2D232B7009
:1028F00001340135381C0A2102F07EFA303129708A
:10290000601CF8BDF7B5089F1E1C051C013A3B0969
:1029100001D1041C05E00093331CFFF7F3FF2C18D2
:1029200006E0601B002A03DD2170013A0134F8E75C
:102930000F231F40092F01D8303704E0002E01D0AB
:10294000373700E0573727700130FEBDF0B585B04E
:10295000041C029101D0002101700025117800298A
:1029600006D1029F0023BD426CD22370281C6FE069
:10297000029FBD42F5D2252902D00132217004E028
:102980005178252904D12170023201350134E5E75F
:10299000302902D0561C202100E0961C32782D3AB6
:1029A00050424241B6180022307830277F423F180B
:1029B000FFB2092F07D80A277A438218D2B2303AD9
:1029C000D2B20136F0E7AF18BC46029FBC4501D930
:1029D0007A1BD2B2692818D00BD863282AD0642871
:1029E00013D0582832D11F1D1B68201C00930123CF
:1029F0001DE075280FD0782814D0732826D11F1D0C
:102A0000201C1B68FFF708FF0AE01F1D201C1B6825
:102A1000FFF73FFF04E01F1D201C1B68FFF713FF9B
:102A20003B1C0BE01F1D1B68201C00930023FFF7BD
:102A300069FFF5E71868043320700120721C241820
:102A40002D188BE7013C2370681E01E001204042F5
:102A500005B0F0BD10B50C1C131C6421221CFFF73F
:102A600075FF10BD00B5031C9BB00A1C01A8191C02
:102A7000FFF7F0FF632800DDFEE701A800F0B6F8DD
:102A80001BB000BD0FB407B504A908C9181C0191FB
:102A9000FFF7E8FF03B008BC04B018470EB403B555
:102AA00003AA08CA191C0192FFF7D4FF02B008BCA0
:102AB00003B0184730B50C1C044303232340041C07
:102AC000002B01D0002310E0032AFBD9CC58C450BE
:102AD0000433D41A032CF9D8131F9B0801339B002D
:102AE000C418C91803231A40ECE7934203D0CD5C05
:102AF000E5540133F9E730BD30B5031C840701D13B
:102B0000032A01D89A1814E00B060C041D1C254357
:102B10000D430C022543031C20C38418E41A032C24
:102B2000FAD8131F9B0801339B000324C3182240CB
:102B3000E8E7934202D019700133FAE730BD021C76
:102B4000031C981A0133591E09780029F9D17047DE
:102B5000031C0A781A70002A02D001310133F8E709
:102B6000704730B50023934208D0C45CCD5C651B30
:102B700006D10133002CF6D1201C02E0002000E039
:102B8000281C30BD10B50022835C8C5CA34204D1AC
:102B90000132002BF8D1181C00E0181B10BD0000FA
:102BA00008B5094BFA211868890002F02FF9FFF7E0
:102BB00031FB96200002FFF77DFD0120FDF742FB6F
:102BC000FEF746FF08BDC0468805001008B5FEF7B1
:102BD000C7FFFFF7FDF8FFF7A5F9FEF785FBFEF746
:102BE00071FBFFF7DDFFFFF7EBF808BD10B5041C24
:102BF0002078002803D00134FDF774FBF8E710BDFE
:102C000038B5051C0E24013C04D3295D0248FFF7AA
:102C100039FFF8E738BDC046EC59000038B519480F
:102C2000FFF730FF184C201CFFF7EAFF174D422139
:102C3000281CFFF727FF201C0E30FFF7E1FF432180
:102C4000281CFFF71FFF201C1C30FFF7D9FF10487E
:102C5000FFF718FF201C4630FFF7D2FF0D48FFF7A3
:102C600011FF201C2A30FFF7CBFF281C4E21FFF755
:102C700009FF201C3830FFF7C3FF616D0648FFF7DE
:102C800001FF38BDEF590000C4050010F5590000E0
:102C9000FC590000025A0000085A000003110A22E1
:102CA00053430F2210401818704738B50A21041CEE
:102CB00002F0ACF80A210501201C02F0FDF8281CE6
:102CC000084338BD08B5C12252000E200221FEF78C
:102CD00019FE024B01225A7108BDC046B80500100A
:102CE00010B5084C6379002B01D1FFF7EBFF237976
:102CF0000C221A43A37901205B001A43011CFEF742
:102D000001FE10BDB805001010B5074C2379002B4B
:102D100008D16379002B01D1FFF7D4FF0123237180
:102D2000FFF7DEFF10BDC046B805001008B5054B23
:102D30001A79002A05D000221A711A72DA70FFF788
:102D4000CFFF08BDB805001010B501210220FEF725
:102D500017FE064B041C18787F231840FFF79EFFD0
:102D6000034B5870DC71201C10BDC0469405001048
:102D7000B8050010014B01229A707047B805001089
:102D8000024B00229A701A727047C046B8050010B4
:102D900008B5FFF7D9FF094B094A9978002908D0EF
:102DA000197A012901D8013103E01068054908604A
:102DB00000E019720021D970116008BDB80500103B
:102DC0006C0300107003001008B5FEF71FFE0C2303
:102DD000184003D0024B1A781043187008BDC04643
:102DE000B805001010B5FFF7EFFF054B1A781C1C53
:102DF000530701D5FFF7CCFF0023237010BDC04659
:102E0000B805001008B50020FEF7E6FB002801D049
:102E1000FFF7E8FF08BD000010B5054C0023E37183
:102E2000FFF7F0FFE379002B01D1FFF78DFF10BD15
:102E3000B805001008B50948092102F049F8084B07
:102E4000FA22D2001A80FFF7E7FF064B00221A6031
:102E5000FA22054B92001A6008BDC046B805001062
:102E6000C20500106C0300107003001008B5FFF7D6
:102E7000C9FF002008BD08B5FFF758FF08BD0000D6
:102E800070B51D4C061C637822781B021343A27890
:102E9000A07912041343E2780D1C12061343174A5B
:102EA00013401A0A237062701A0C1B0EE3706379C8
:102EB000A27022791B021343114A134023711B0A8B
:102EC0006371FFF7EBFE0F4B1B88C01830806079F1
:102ED000FFF7E4FEB070E078FFF7E0FEF070A07856
:102EE000FFF7DCFE28706078FFF7D8FE6870207866
:102EF000FFF7D4FEA87070BD940500107F7F3F3FA0
:102F0000071F0000C2050010F0B58DB0051CFEF7CC
:102F100047FD002804D1281C1249FFF7BFFD1EE021
:102F20000AAE0BAC211C301CFFF7AAFF3388F778E0
:102F30000793B378267808936378A47809930A4BAB
:102F4000187900F0D7F8099B049002930097019636
:102F50000394281C0549079A089BFFF79FFD0DB0B5
:102F6000F0BDC046145A000094050010195A000024
:102F700070B5061C0D1C141CFEF712FD00280AD0AB
:102F8000301C291CFFF77CFF002C07D0044B0020CD
:102F90001B79236003E00120404200E0201C70BD4B
:102FA00094050010F7B504880E1C051C6421201C34
:102FB0000092019301F020FF114B8FB2B078E41B17
:102FC0001C80FFF772FE0F4CA0707078FFF76DFE4B
:102FD000E0703078FFF769FE2071E878FFF765FE52
:102FE000009B6071A371A878FFF75FFEE071381C49
:102FF000FFF75BFE20720198FEF7E4FCFEBDC046C1
:10300000C2050010A405001008B50223FFF7CAFF8F
:1030100008BD08B5021C501E82415201002001214A
:10302000FEF770FC08BD38B5041C01200D1CFFF72D
:10303000F0FF201C00F086F8072101F03DFF201C66
:103040000A1C291CFFF7E0FF96204000FFF7FCF860
:103050000020FFF7DEFF38BD73B5041CFFF774FED8
:10306000002801D100203BE01E4B5D781E1C7378C8
:10307000AB4207D10A20FFF7E7F8FFF765FE00280B
:10308000F5D1EFE7FEF78CFC0028EBD001A96846EC
:10309000FFF7F6FE684600F055F8051C01A800F0A1
:1030A00031F8114B04199C420DD9E3170122134347
:1030B000ED18281C694600F075F8002C01DA0B4B5E
:1030C00000E00B4BE418201C01A900F024F8281C98
:1030D000072101F0F1FE68460A1C01A9FFF794FFE1
:1030E00076BDC046B80500107F5101008051010037
:1030F00080AEFEFF07231840014B8000C058704788
:10310000EC00001002783C235A4341785218534394
:1031100082789818704738B50C1C3C21051C01F0CA
:10312000CBFE281CA1703C2101F070FE3C2101F077
:10313000C3FE6170E121281C090101F067FE2070C7
:1031400038BD000070B583780221002299425241B7
:10315000048896214901051C64180C20A41A4243D6
:103160009B18033B992058430521023001F04EFE85
:103170006E26FF3666436421A31086194942201C3F
:10318000F61801F043FEC82136184900201C01F052
:103190003DFE034B3018C018EB78C01870BDC04618
:1031A000D382FFFFF8B5204B0C1CC5181F4B8000C5
:1031B000C0181F4901F02AFE03235843C617B60F53
:1031C0003618B610AE19B600953E301C194901F0FC
:1031D00073FECD17AD0F6D180527AD107D43023579
:1031E000281C992101F068FE081C391C01F00EFE14
:1031F0000130E0709921281C01F008FE0C210230FA
:1032000001F05AFE4D1CEDB2A570301C094901F0C9
:10321000FDFD094B0C21C6180E20401B01F0F6FDE8
:1032200036182680F8BDC04679050000652F0400D9
:10323000B13A0200B505000094EDFFFFF8238A01C2
:10324000DB0013404A05920E1343F822120211408C
:1032500019430A23594330B5CA1083181C1CEB3498
:103260005D782478EA336C401B7824021C43835C2D
:10327000201C58400723194008418005800D30BDAF
:103280007047000008B5054B011E994201DD044B53
:10329000C1180448EA38FFF7D1FF08BDFF17000046
:1032A00000F8FFFFA75A00000723594310B5084B49
:1032B00059189C310023CC5C0F2222400270CA5C5A
:1032C0000133120942700230072BF4D110BDC04601
:1032D000C40500100723594310B5074B59189C31FA
:1032E00000234278047812012243CA540133023089
:1032F000072BF6D110BDC046C405001070B5AD4C0B
:1033000086B0E36E6E465A1E934117363370AA4B51
:103310009A6A191CD006400F0138062807D801F018
:1033200013FD040C2012181A1D00022509E0636E1B
:1033300016339B001B591D1C15E0636E16339B0052
:10334000E55800230FE0A36DE56DAB420BDD0D25C5
:1033500009E0022503E00C25032304E00D252B1CC6
:1033600001E00D25EDE70D6150111F2800D91BE18B
:1033700001F0F4FC2000220029002C002F00330073
:103380003B00440048004C00540061006E00760091
:1033900083008F009B00A800B800C500D500D300B3
:1033A000E100E400E700EF00FE0002010B010D0167
:1033B0000F011501E01801E0E0180E30EB1A591C5E
:1033C00001F086FDF0E0E0181C30F7E7211C0E311B
:1033D00005E0E0180E30E1180BE0211C1C31201C28
:1033E0001A1C2B1C01F0EDF8DEE0E018E1181C308F
:1033F0000E31EB1A5A1CFFF75DFBD5E06F48011C3C
:103400000E31EDE7E018011C1C31F2E7226E1021AD
:10341000002A00D00A21221C0E3206E0226E102162
:10342000002A00D00A21221C1C320291009501962C
:10343000201C211C53E0216E012232701022002931
:1034400000D00A22009501960292201C211C45E022
:10345000226E1021002A00D00A21221C0E3213E015
:10346000216E012232701022002900D00A2200951C
:1034700001960292201C211C4DE0226E1021002A90
:1034800000D00A21221C1C32009501960291201CBA
:103490006AE0226E1021002A00D00A21484A0291D7
:1034A00000950196101C111C19E0216E10200029B6
:1034B00000D00A20424A0290111C1C390095019646
:1034C000101C0CE0216E012232701022002900D065
:1034D0000A223B49009501960292081C002201F045
:1034E0007AF861E0226E1020002A00D00A20344AC7
:1034F0000290111C1C3900950196101C35E0216EBC
:10350000012232701022002900D00A222C49009595
:1035100001960292081C002227E001223270226EDE
:103520001021002A00D00A21254A02910095019617
:10353000101C002119E0009620481BE0009620484E
:1035400018E0226E1021002A00D00A21221C1C3211
:1035500006E0226E1021002A00D00A21221C0E3221
:103560000095019602910020211C01F05CF81BE0FF
:103570000096201C002103E0211C1C310096201C19
:103580001A1C2B1C01F0ACF80EE0201C02E00B48CA
:1035900000E00B48191C2A1C01F0B9F804E0201CBB
:1035A000191C2A1C01F0BDF833780120E36606B02F
:1035B00070BDC046C4050010600D0010D20500109B
:1035C000E0050010064910B50A1C883213681C1C5F
:1035D0001E34A4006050013303210B40136010BD62
:1035E000C4050010054B0322191C883108680138F6
:1035F00002400A601E329200D0587047C405001085
:10360000F7B5124F3D1C8C3528680130FFF73AFEA4
:103610000F4EBB6EB26A041C01920122F06202409E
:103620009A4210D1830703D428680230FFF7CAFFFB
:10363000FF239B00019A1C40A40193101C438C376C
:1036400001233C60F3600220FEBDC046C4050010AB
:10365000600D00100C490D488A6A031C8C3370B54C
:103660001D68D3059B0E0C1C910500D5403B866E52
:10367000921001210A40B24203D18C30EB18036052
:10368000E160012070BDC046600D0010C40500104F
:1036900008B5084B5A1CD07F9A1CD27F0001120239
:1036A000104303331A7FDB7F10431B031843FFF7DC
:1036B00089FF08BDC405001008B5FFF793FF032379
:1036C000044A0F219A180140013311770011072B8A
:1036D000F6D108BDC405001008B5FFF783FF034B02
:1036E00001228C331860024BDA6008BDC40500105B
:1036F000600D001010B5064CA36E002B06D0FFF72E
:1037000071FF044B8C3401222060DA6010BDC0468A
:10371000C4050010600D001010B5064CA36E002B00
:1037200006D1FFF75FFF044B8C3401222060DA6082
:1037300010BDC046C4050010600D001008B5104B48
:103740000022596A1A62914214D05969914216DDD9
:10375000012906D1D969914203D0DA610A2299611F
:103760005A615A69032A02DD06490120C866013AF6
:103770005A6104E0044B1B68002B00D0984708BD39
:10378000600D0010C405001034040010074B5A6A85
:10379000002A02D05A69002A07DD9A690F21044BDA
:1037A0001140D97712110133DA777047600D00109C
:1037B000C4050010044B597F9A7F090112020A4385
:1037C000197F0A435A677047C40500100B1C093B58
:1037D00010B5012B0FD80023074A9A18147FC25C3A
:1037E000944205D0054B08395A681143596002E0EC
:1037F00001330E2BF0D110BDC4050010600D001078
:1038000008B508290DD0192913D1427808231A4286
:1038100002D00022027002E00F23037007234370DE
:1038200005E000230022C25401330E2BFAD1FFF72A
:1038300051FD08BD30B5114D85B06C6F002802D028
:103840000F239C4304436C67FF2C05DD281C1C30B0
:103850000E2101F03DFB0FE06846211CFFF724FD1F
:103860006846211CFFF7CCFF00236846C15CEA18BC
:10387000013311770E2BF8D105B030BDC40500100F
:10388000134B30B5596F0F229143041C0C4385B084
:103890005C671D1C082C19D0FF2C17DC6846211C06
:1038A000FFF702FD6846211CFFF790FF0023EA188E
:1038B000127F6946CA5401330E2BF8D16846211C89
:1038C000FFF79EFF6846211CFFF704FD05B030BDE1
:1038D000C40500101FB50F4C616F082918D0FF29CF
:1038E00016DC6846FFF7E0FC6846616FFFF76EFF85
:1038F0000023E218127F6946CA5401330E2BF8D117
:103900006846616FFFF77CFF616F6846FFF7E2FC76
:103910001FBDC046C405001010B50D4C631CD87FF8
:10392000A31CDB7F00011B021843E37F1843E31C49
:10393000DB7F1B031843FFF7A5FC0F23021C1A4073
:1039400022770211134000126377A07710BDC046A2
:10395000C4050010044B5A6E16329200D258121A47
:1039600051424A41DA667047C4050010044B5A6E52
:1039700016329200D158013900D50D21D15070472F
:10398000C4050010054B5A6E16329200D158013111
:103990000E2900D10021D1507047C046C405001047
:1039A000094B5A6E16329200D2580D2A03D11A1CB6
:1039B0002932127805E09A18507F117F0001021C0D
:1039C0000A435A657047C046C4050010084B10B53D
:1039D0005A6E0F2416329200D1585A6D581814405E
:1039E000013104770D2902DC5B1812111A7710BD22
:1039F000C40500100E4B30B55A6E596D1632920048
:103A0000D2580D2A07D11C1C2934F02024780840F4
:103A10002043586507E09818447F057F24012C4314
:103A20005C650C1144779B180F221140197730BD4B
:103A3000C405001008B503480E22011C1C39FFF70D
:103A400039F808BDFC05001008B503480E22011C1A
:103A50001C31FFF72FF808BDE005001008B5044839
:103A60000022011C1C310D2300F0ABFD08BDC04637
:103A7000E005001008B503480E22011C0E39FFF7BF
:103A800019F808BDEE05001008B503480E22011C08
:103A90000E31FFF70FF808BDE005001008B5044827
:103AA0000022011C0E310D2300F08BFD08BDC04625
:103AB000E00500100023044A00219A184632013321
:103AC0001170082BF7D17047C4050010C31C421EAB
:103AD0000020934207D00449400059184631097824
:103AE000013B0843F5E77047C405001010B50B1DF6
:103AF000994208D0044A01248A18044046321470BE
:103B000040100131F4E710BDC405001038B50020A5
:103B1000FFF7DCFF084C051C0021207FFFF7E6FFC4
:103B200004202577FFF7D2FF0421051C607FFFF7F3
:103B3000DDFF657738BDC046C405001010B5002014
:103B4000FFF7C4FF034C20770420FFF7BFFF607727
:103B500010BDC046C405001010B5054C0021207FE3
:103B6000FFF7C4FF607F0421FFF7C0FF10BDC04610
:103B7000C405001010B5094C231C8C3318680130A3
:103B8000FFF780FB064B021CD8620F231A402277F6
:103B90000211134000126377A07710BDC405001016
:103BA000600D001010B5084C0E21201C01F090F99A
:103BB000201C0E300E2101F08BF9201C1C300E2130
:103BC00001F086F910BDC046C405001010B50C4BBD
:103BD000191C0E311A1C187F1C7801332043D8762B
:103BE0008B42F8D1936E002B08D0064B1B690D2B2E
:103BF00004D1137F111C29310B70537310BDC046C3
:103C0000C4050010600D001010B50C4B191C0E31CE
:103C10001A1C1C7F187801332040D8768B42F8D1CB
:103C2000936E002B08D0064B1B690D2B04D1137F1C
:103C3000111C29310B70537310BDC046C405001010
:103C4000600D001030B5002185B00E4B421C1818D5
:103C5000007F6C4608550D25D40F181C0023954293
:103C60005C416442013122400E2901D0101CECE776
:103C70006C46E15CC218013311770E2BF8D105B008
:103C800030BDC046C4050010074B10B55A6E163241
:103C90009200D458611E1C19D1502077002901DAF6
:103CA0000D21D15010BDC046C4050010034A0023A9
:103CB000111C943198320B6013607047C4050010DA
:103CC000034B0122943319684A401A607047C0467A
:103CD000C4050010044A002313678C321360034BA1
:103CE0000122DA607047C046C4050010600D001064
:103CF00010B59E4C0F20A16A9D4A8B101840891167
:103D0000013852560E2848D801F01EF8080F171F28
:103D1000234729474731474747353900002A3CDBCD
:103D2000944B9A184032002305E0002A35DB914B72
:103D30009A184032012393712DE0002A2DDB8D4B20
:103D40009A1840329279DA6625E0081CFFF79CFF4A
:103D500021E0002A21DB101CFFF7FCFD1BE0002AFC
:103D60001BDB844B596E16318900CA5013E0081CC6
:103D7000FFF786FD0FE0081CFFF75CFD0BE0002A53
:103D80000BDB101CFFF75EFF05E00C2B23DD162B71
:103D900028D1FFF705FE0120EEE0982B03D1754BEB
:103DA00000221A66F7E7982B6CDC382B03D1714B95
:103DB00001205866E0E0382B30DC1C2B02D1FFF7E5
:103DC00039FEE8E71C2B12DC0C2BDED1694B0120FD
:103DD00098331860D0E00120002B00D1CCE0012006
:103DE0004042C9E0182BFAD1FFF774FFD3E7282B24
:103DF00003D1604B00225A66CDE7282B04DC262B2A
:103E0000EDD1FFF7E3FDC6E72C2B02D1FFF71CFE37
:103E1000C1E7362BE3D1FFF7EDFDBCE7662B02D1FE
:103E2000FFF732FEB7E7662B16DC4C2B03D1FFF70A
:103E3000A1FE0220A0E04C2B04DC3C2BCFD1FFF7ED
:103E40000DFEA8E7562B02D1FFF714FEA3E75C2B6B
:103E5000C5D1FFF71DFC9EE76C2B02D1FFF72CFCB0
:103E600099E76C2B04DC682BB9D1FFF79BFE92E736
:103E7000762B02D1FFF712FE8DE7882BAFD1FFF72B
:103E800085FC88E7E62B02D1FFF758FE83E7E62B97
:103E900035DCC82B02D1FFF713FF7CE7C82B16DCFB
:103EA000A82B03D1334B0120186665E0A82B04DC56
:103EB0009C2B94D1FFF77EFC6DE7B82B02D1FFF766
:103EC000F5FE68E7BC2B8AD1FFF704FD63E7D62B2C
:103ED00002D1FFF741FE5EE7D62B05DCCC2B00D0EC
:103EE0007DE7FFF719FD56E7D82B02D1FFF702FC5B
:103EF00051E7DC2B00D072E7FFF768FE4BE7F32BAE
:103F000002D1FFF71BFC46E7F32B17DCEC2B02D1A9
:103F1000FFF77AFE3FE7EC2B05DCE82B00D05EE7ED
:103F2000FFF7FAFB37E7F12B02D1FFF7C3FD32E7CA
:103F3000F22B00D053E7012020621DE0F62B02D1C6
:103F4000FFF7E4FD27E7F62B05DCF52B00D046E76D
:103F5000FFF70CFD1FE7F72B02D1FFF713FD1AE760
:103F6000F82B00D03BE7FFF7B7FB14E7600D00101C
:103F7000A7960000C405001010BDC04638B5184C07
:103F8000231C8C331868FFF77DF9164B0022E16E75
:103F9000DA60E26603229862A16610401D1C0228C6
:103FA00009D090420AD0012802D0FFF7A1FE07E015
:103FB000FFF726FB04E0FFF7A1F901E0FFF74AFB5A
:103FC00000280BDDEB68002B04D1231C8C3319680F
:103FD0000A181A60903422681318236038BDC0464E
:103FE000C4050010600D0010034B0122DA660F2299
:103FF0009A775A771A777047C405001010B5054CA8
:104000000549201C00F064FFFFF7EEFF0123636603
:1040100010BDC046C40500109C070000704700009A
:1040200030B50C4D049C28600B4801600B490A60B8
:104030000B4A13600B4B039A1A600B4B0B4A1C6024
:104040000B4B1C600B4B1A600B4B0C4A13600C4A59
:10405000136030BD58040010640400106C0400109C
:10406000400400103804001010010010C54000008A
:10407000600D0010340400101D40000068040010A2
:1040800050040010014B18607047C0463C040010FB
:10409000094B10B51A68191C084B002A03D1084CAB
:1040A0002468226003E01A68904200DA101C18604D
:1040B00001230B6010BDC0464404001060040010D2
:1040C0003C04001013B5002300930193114B124CD4
:1040D0001A68124B11681868814202D12268009256
:1040E00008E012681A600E4B1B68002B02D068466D
:1040F00001A99847009B2360002B04D0094A642043
:104100009361FFF7C5FF009A531E9A41064BDA668A
:1041100013BDC04640040010540400100C010010F0
:1041200064040010600D0010C4050010034B1B68F0
:10413000002B01D1024A13607047C0464C040010A6
:1041400044040010014B4A3318787047C40500102E
:1041500038B5164B1A1C98321268002A04D0144B3A
:104160001C6801231C4001E094331C68114DAB68AE
:104170009C4202D16A68002A16D0002C02D1002B82
:104180000AD111E00C4B1B68002B02D0201C69687F
:10419000984700236B6006E0074B1B68002B02D09A
:1041A000201C211C9847AC6038BDC046C4050010D7
:1041B00048040010600D00105804001008B5084AAB
:1041C000084B126819688A1A05D5FA2252001A603B
:1041D000054B1A6801321A60FFF7BAFF08BDC046E6
:1041E000380400101401001048040010F8B50E1C2B
:1041F0000E21041C171C00F06BFE174B03259E427A
:1042000011DD092363730123237323E0301C0A218A
:1042100000F052FE301C61550A2100F0F7FD013517
:10422000061C0D2D01D0002EF0D1EF1B033F27708F
:104230006B1E022B05D0E15C621BD2185173013B4F
:10424000F7E70F235D1B013D6B1C032B02DD0023F1
:104250006355F8E7F8BDC046FFC99A3B37B5041C63
:104260000025002300930193124B1B68002B02D002
:10427000684601A9984700980135002800D000251C
:104280000220FCF75CF80C4B1A680C4B116818689C
:1042900081420AD012681A60FFF790FF002C04D008
:1042A000013C002C01D1201C02E0032DD9DD0120AE
:1042B0003EBDC04664040010400400105C040010C1
:1042C000F7B59B231E4A5B000D1CD45C38213023BC
:1042D000FF33FF31D35C515C161C002C02D00F223F
:1042E000114002E08024072164009A225200B75C4A
:1042F0003622FF32B25CE31ABA1A80277F003C1BD9
:1043000000940724611A019101320E490024FEF73E
:10431000C5FB2C70281CFEF712FC34273119FF371F
:10432000CB193531FF311F780B784122121B281829
:10433000FB1A0549013CFEF7B1FB631DEAD1F7BD4D
:10434000C4050010B7960000C4960000F0B5544DA7
:10435000544C2B1C94331B6893B0061CA061E16184
:10436000002B17D118280BD1C32909D14E4B1B683C
:104370000F2B05D1281C38300E21162200F00CF925
:10438000A069182804D1E269332A01D100F0AAF803
:10439000FFF72AFE002E02D00A23636100E0666167
:1043A000424BA069424F18603B68424E1B68336025
:1043B000FFF7BCFE012300222B6701923E4B1B68D6
:1043C000002B1AD03D4E3368371C002B15D01B68CC
:1043D000002B04D13A4B1B6898473B68F7E73368DA
:1043E0001A68013A1A60374A1368002B05DD013B51
:1043F0001360002B01D1FFF799FEFFF7BFFD0028E6
:1044000001DAFCF74BF8019A40239A432E4B9A426B
:1044100008D1A26A10239A432C4B9A4202D10A2057
:10442000FFF736FEA36A2E1C8C360193284A3368A8
:10443000934203D0274A93420BD019E0FFF788FE3E
:10444000FBF7ACFF1B481B4A0068031C013B1360D1
:104450000EE0214F3B68002B0AD002A80AA9FFF703
:104460002FFF3B6802A80AA99847336827333360B7
:104470001A4B1B6898470E48194B02681868116858
:10448000814206D012681A60FFF798FE0C4B1B6839
:1044900098472A6F002A91D1FFF75AFE13B0F0BD5A
:1044A000C4050010600D001010010010540400102D
:1044B000400400100C010010440400103C040010E3
:1044C000680400106004001026020000EB030000E6
:1044D000790D00003E2700006C040010500400100D
:1044E0005C040010F7B5274E002033681C68FFF706
:1044F000B5FE33681A689442FCD01B6801272D333F
:10450000FF330193FFF770FD1F4C0A231F4D6361BA
:104510001823A3611523E3612B1C903300226762EB
:104520001A60FFF761FD2F673368019A1B689A4292
:104530000CD0FFF723FD3268154B116818688142D3
:10454000F2D012681A60FFF739FEEDE72B1C012745
:104550009033182000211E686762FFF7F7FE0D4BAD
:10456000301C196800F052FC3835011C0422281C4C
:10457000FFF73CFE1823A3610023301C6762E36150
:10458000FEBDC04640040010600D0010C4050010C0
:104590005C0400103804001070B5002A10DD0478A7
:1045A00001231C404B1E002B08DBC55CE4006E0899
:1045B0003443C4540124013B2C40F4E7013AECE7B6
:1045C00070BD30B59A4205DC845C8D5C85548C549A
:1045D0000132F7E730BDF0B5069E051C07A8047848
:1045E0003078002A17D0059EB34217DCCE5CD75C2A
:1045F000F7193F180020A74201DB3F1B0120EF54B1
:104600000133F0E7CA5C12180020A24201DB121B42
:104610000120EA540133059A9342F3DD0123184047
:10462000069B1870F0BDF7B50AAC2478099D00947C
:10463000089E2C7800282DD0002928D0002A18D0D8
:10464000B34248DCCF5CD55C7F1B3F1B0024A742F4
:1046500002DA009C3F190124C7540133F0E7CA5C19
:10466000121B0024551C02D1009A0124013AC254A5
:104670000133B342F3DD2EE0D15C4942091B002433
:10468000A14202D0009F0124C919C1540133B34291
:10469000F2DD20E0002914D0002A08D0B3421ADC51
:1046A000CD5CD05C0133281A041BE40FF6E7B3425B
:1046B00011DCCA5C0133141B013462425441E4B280
:1046C000F5E7B34207DCD15C013349420C1B611EA4
:1046D0008C41E4B2F5E701231C40099B1C70F7BD37
:1046E00070B5049C0125257000290BD09A420BDC83
:1046F000865C8D5CAE4209D10132F7E7815C00290E
:1047000004D101329A42F9DD0023237070BD914239
:1047100004DA43185B7843540131F8E7002343542B
:1047200070478A4205DD8318013B1B788354013AA8
:10473000F7E7002383547047F7B5134A134C1378F7
:104740005278C35C134000D04023114923601231DA
:10475000009100220023A6187360009B0125123BE4
:104760001F785978C75D394202D077682F43776048
:10477000009F02336D00BB42F2D11233043200932A
:10478000282AE7D10020FEBD0D020010200F0010E6
:1047900059010010122330B54B43334A0131D3186D
:1047A000052251431A785C78825C144204D02F4A67
:1047B0005F245218947054709A78DC78825C1442AA
:1047C00004D02A4A7C245218533214701A795C7926
:1047D000825C144204D0254A7C245218A3321470FF
:1047E0009A79DC79825C144207D0204C5F226418ED
:1047F000251CA235A1342A7022701A7A5C7A825C58
:10480000144204D0194A7C245218A03214709A7AA7
:10481000DC7A825C144204D0144A7C245218503250
:1048200014701A7B5C7B825C144207D00F4C5F22B1
:104830006418251C523551342A7022709A7BDC7B17
:10484000825C144204D0094A2E245218A4321470F7
:104850001A7C5B7C825C134204D0044B5918F431FF
:1048600027230B70002030BD59010010900D00105F
:10487000F8B52E4D061C00272C1C281C20214F2289
:10488000FEF73AF9002F04D02A1C7C2339322B7012
:1048900013702B1C4F33002201371A705035052F2F
:1048A000EBD1211C2D2338310B70211C37310B70BB
:1048B000A121A370637049005F2363544221FF313B
:1048C0006354A32149006254194A11785278715CEB
:1048D0000A4204D0221C5332523413702370002435
:1048E000211C301C0134FFF755FF0A2CF8D100249D
:1048F000104B114DE25C1B19B15C58780F4A6300F4
:10490000084201D0D15805E0D058FEF718F90C49FB
:10491000091A0A31281C023400F0E4FA122CE7D1FB
:10492000281C084900F0DEFA0520F8BD900D0010A3
:104930000D02001018010010D00E00102C01001004
:104940000F020010CC960000F0B585B00190FCF786
:10495000B9FCA24CA24F00260C257543002E00D1B5
:104960000125A04B1B68012B02D0022B10D001E0C7
:104970009B4F0EE0002B0CD12168C90700D4ACE09E
:10498000681CC0B2002107220223FCF713FDA4E03B
:10499000954F002303A8437023687F2213405C2BAC
:1049A00000D191E027DC382B00D187E011DC072B08
:1049B00065D005DC022B00D18DE0062B40D0DBE773
:1049C000212B00D17EE0232B00D181E01C2BD3D101
:1049D0007CE04F2B4DD007DC3F2B61D0402B61D0CA
:1049E000392BC9D1432374E0542B71D05B2B3ED0BB
:1049F000502BC1D166E0732B62D00FDC662B3AD00E
:104A000004DC5E2B52D0622B60D0B5E76F2B3AD01E
:104A1000712B4FD06D2BAFD135235AE0792B47D076
:104A200006DC762B48D0772B3ED0742BA4D143E004
:104A30007D2B22D07F2B24D07C2B9DD1422348E09C
:104A400031230370022E00DCDCE0231C083B1B68D2
:104A50001A40542A32D0032E00D1D3E0231C0C3B41
:104A60001A687F231340542B00D0CBE026E032237A
:104A70002FE033232DE034232BE0362329E03723A6
:104A800027E0382325E039230370062E00DCB9E047
:104A9000231F1B681A404723232A00D0B2E018E0E6
:104AA000302316E02D2314E0412312E0442310E0CC
:104AB00045230EE046230CE048230AE04C2308E09F
:104AC000502306E0522304E04F2302E0552300E088
:104AD0004E23037096E04923FBE72168022211422E
:104AE00005D0A81DC0B200210623FCF763FC236893
:104AF00004210B4205D0A81DC0B202220623FCF7F8
:104B000059FC236808210B4205D0681CC0B207225B
:104B10000223FCF74FFC2168C90606D5681CC0B209
:104B2000042102220623FCF745FC23689B0606D5D8
:104B3000681CC0B2002102220623FCF73BFC21685E
:104B4000490606D5681CC0B2042107220223FCF7DF
:104B500031FC23681B0607D5281C09300222C0B28D
:104B60000821131CFCF726FC2168C9050BD5EDB202
:104B7000281C0930C0B20B210A35FCF707FCE8B24B
:104B80000A21FCF703FC013604340B2E00D0E3E6C7
:104B9000164B1B68002B05D0154800210922154B28
:104BA000FCF77EFC144D00240235AB1E1A780199E7
:104BB0006B1E8A5C1B78134208D0104BA200D058A1
:104BC0000F4B0922E15C0B4BFCF76AFC0134023508
:104BD000092CEAD1FCF780FB05B0F0BD200F0010D6
:104BE000080000101C020010000000104C02001011
:104BF000D6960000140000101801001020020010CA
:104C0000500100103B1C291C0022FCF749FC2368C2
:104C10001B0605D5E91D074800223B1CFCF740FC9C
:104C20002368DB05AFD5E91D034800223B1CFCF7D8
:104C300037FCA8E717590000D496000038B5FFF7F5
:104C400081FA0624002805D1FCF746FB38BD013463
:104C50000E2CF9DC0321201C00F0D8F80321C5B28A
:104C6000201C00F029F9281CC9B2FCF78FFB092C85
:104C7000EDD10B24EEE7000038B5041CFFF75CFD16
:104C8000201CFFF761FE094B1B78002B0DD0201C68
:104C9000FFF7EEFD064CC8235B00E518211C054814
:104CA0005034FDF7EFFEAC42F8D138BD7804001067
:104CB000900D00105650000000B589B000280ED0AD
:104CC000FCF7CBFA01A80921FEF7EEFA684612308C
:104CD0000A21FEF7E9FA01A8FFF7CEFF08E0FCF78A
:104CE000C4FA044B1B78002B02D00348FDF7CAFE20
:104CF00009B000BD78040010D8960000FEE7FEE77A
:104D000008B500230B4A0C499A188A4204D20B4971
:104D1000C95C01331170F5E7094B0A4A591C013B84
:104D2000934203D200221A700B1CF6E7FBF758FFE0
:104D3000FEE7C04600000010440200102F9700005C
:104D4000450200104C0F001002B47146490849009A
:104D5000095C49008E4402BC7047C04603B47146EA
:104D6000490840004900095A49008E4403BC704775
:104D7000002934D00123002210B488422CD301240E
:104D80002407A14204D2814202D209011B01F8E7A3
:104D9000E400A14204D2814202D249005B00F8E75C
:104DA000884201D3401A1A434C08A04202D3001B88
:104DB0005C0822438C08A04202D3001B9C082243BB
:104DC000CC08A04202D3001BDC082243002803D0F9
:104DD0001B0901D00909E3E7101C10BC704700282B
:104DE00001D00020C04307B4024802A1401802903D
:104DF00003BDC046D90000000029F0D003B5FFF77D
:104E0000B9FF0EBC4243891A1847C046002941D059
:104E100010B4041C4C40A44601230022002900D5F4
:104E20004942002800D5404288422CD3012424075F
:104E3000A14204D2814202D209011B01F8E7E40039
:104E4000A14204D2814202D249005B00F8E78842C5
:104E500001D3401A1A434C08A04202D3001B5C083D
:104E600022438C08A04202D3001B9C082243CC089A
:104E7000A04202D3001BDC082243002803D01B09F8
:104E800001D00909E3E7101C6446002C00D540421C
:104E900010BC7047002806D003DB0020C043400848
:104EA00001E08020000607B4024802A140180290E9
:104EB00003BDC046190000000029EBD003B5FFF781
:104EC000A7FF0EBC4243891A1847C0467047C04628
:104ED00042180023002903D0037001309042FBD117
:104EE0007047C04670B5061CB30717D133680F482A
:104EF0000F4D1A189A43301C2A420FD10430026811
:104F00000A4BD41894432C4208D104300268074B52
:104F1000D41894432C42F1D000E001300278002AEA
:104F2000FBD1FDF715FE301C70BDC046FFFEFEFE36
:104F30008080808025732025730D0A00444D313513
:104F40005F4D31420053455249414C20434F4E532F
:104F50004F4C45007265616479000D0A4279652EF7
:104F60002E2E0D0A004E4F00203F00257320257382
:104F7000202025694D485A005632330020202569EB
:104F80002E253033695600202573525443200044A7
:104F90004D343100444D3431204F4B0020204552D8
:104FA000523A20256900424144204B455920253082
:104FB000327800202D2025303278004C43443A25A9
:104FC000303269202D202569005052455353204529
:104FD0004E54455220544F205341564500256331CD
:104FE00020484F5552002D003A005254432052455C
:104FF0004144204641494C007475726E6564206FCF
:105000006E003C52455345543E0D0A0042616420F7
:105010006E756D6265722E0D0A004241543A20256C
:10502000696D560D0A000D0A253032782020005790
:10503000616974696E6720666F7220646174612EA5
:105040002E2E0D0A00426164206D6F64656C0D0A9E
:1050500000526561642025730D0A004641494C45A4
:1050600044006F6666004C434420646562756720A7
:1050700025730D0A00436F6E736F6C652074696D44
:10508000656F75742073657420746F202569206DB9
:10509000696E757465730D0A00000000005C000CF9
:1050A000000C7C287C7C447C241048285408000C8C
:1050B00000384400443800201008103810804000A8
:1050C000101010004000201008384438007C0064A4
:1050D00054484454281C107C4C54243854200474E4
:1050E0000C285428085438005000805000102844E0
:1050F000282828442810045408384C5C7814787CFC
:1051000054283844447C44387C54447C1404384447
:10511000347C107C007C0020403C7C106C7C404047
:105120007C087C7C047C7C447C7C14083844787C3F
:105130001468485424047C047C407C3C403C7C2023
:105140007C6C106C1C601C64544C7C440008102067
:10515000447C0008040880808004080078447800BB
:1051600007080400000000BF01BF01090500000797
:10517000000700070007130A00002000E400FC00FD
:105180003F00E700FC003F002700040F0800000C70
:10519000011E01FF03FF032201E201C2190D0000FD
:1051A0000E001F0011019101FF007E00FC00FE01B6
:1051B00013011101F001E0140A0000EE00FF0111DB
:1051C000011101BF01EE00E00130011001050300F3
:1051D000000F000F0A050000F800FE030707010496
:1051E0000B060000000001040707FE03F80F08008B
:1051F0000000000A000E001F001F000E000A110927
:105200000000100010001000FE00FE001000100052
:1052100010080400000004800780030D0700001040
:105220000010001000100010001008040000000022
:10523000800180010D07000C000FC003F0003C004E
:105240000F00030F080000FE00FF01010101010132
:1052500001FF01FE10080000000002010201FF0131
:10526000FF0100010001100800008601C701610173
:10527000210131011F010E010F080000820083018E
:10528000110111011101FF01EE1109000030003878
:10529000002C002600FF01FF012000200F08000065
:1052A00080009F011F0111011101F101E10F0800B0
:1052B00000FC00FE010B0109010901F901F00F08D2
:1052C000000001000100C101F1013D000F00030FCA
:1052D000080000EE00FF01110111011101FF01EEB4
:1052E0000F0800001E003F0121012101A101FF0064
:1052F0007E0804000000008C018C010804000000FE
:10530000048C078C0312090000200070005000D8A4
:105310000088008C010401040111090000480048C4
:1053200000480048004800480048004811090000B3
:10533000040104018C018800D80050007000200D89
:1053400007000002000300B101B9010F0006190DAA
:105350000000F800FC010603FB06FD050505050538
:10536000FD05FF050601FC01F8120900008001F0AF
:10537000017C004F004F007C00F00180010F08000D
:1053800000FF01FF01110111011F01FE01E01109E0
:1053900000007C00FE008301010101010101830185
:1053A0008211090000FF01FF0101010101010183D8
:1053B00001FE007C10080000FF01FF011101110136
:1053C0001101110111010F080000FF01FF0111007F
:1053D00011001100110001120900007C00FE008381
:1053E00001010121012101E301E20112090000FF95
:1053F00001FF011000100010001000FF01FF010A62
:105400000500000101FF01FF0101010B0600010081
:105410000101010101FF01FF10080000FF01FF0170
:1054200038006C00C6008301010110080000FF0174
:10543000FF0100010001000100010001160B000046
:10544000FF01FF010F003C00F000F0003C000F00E6
:10545000FF01FF0112090000FF01FF010F001C0006
:105460007000E001FF01FF01130A00007C00FE0054
:1054700083010101010101018301FE007C0F08008D
:1054800000FF01FF012100210021003F001E140A3E
:1054900000007C00FE00830101010101010383077C
:1054A000FE047C0412090000FF01FF01210021001D
:1054B0007100DF008E010001110900008E009F01C4
:1054C0001101110111011101F301E21109000001A3
:1054D0000001000100FF01FF0101000100011109AD
:1054E00000007F00FF008001000100018001FF003B
:1054F0007F1109000007001F007800E001E001783B
:10550000001F0007190D00000F007F00F001E001EF
:105510007C001F001F007C00E001F0017F000F12E3
:105520000900008301C7016C00380038006C00C717
:1055300001830111090000010007001E00F801F8B5
:10554000011E00070001120900008101C101610173
:10555000310119010D0107010301000404020000DB
:105560007F0109050000070000000000070B06444A
:1055700000FF0144004400FF01440B0600008C00C2
:105580001201FF032201C40D07820045002500928D
:105590000048014401820C060000E60019012601C2
:1055A000C000200107040000000001000208040000
:1055B000000000FE0101020804000000000102FEDC
:1055C000010B0600008800500020005000880B06E8
:1055D000000020002000F80020002006030000004A
:1055E0000400020B06000020002000200020002004
:1055F00006030000000000010905000080016000B2
:105600001800060B060000FE00010101010101FE69
:105610000804000002000200FF010C0600008201E5
:105620004101210111010E010B0600008200010160
:1056300011011101EE0B060000600058004600FF4A
:1056400001400B0600009F00090109010901F10B4F
:10565000060000FE00110111011101E20B0600001D
:105660000100C10131000D00030B060000EE001126
:105670000111011101EE0B0600008E001101110154
:105680001101FE0804000000008C018C01080400D8
:10569000000000000208010A0500002000500088F8
:1056A0000004010B06000050005000500050005054
:1056B00009050000040188005000200B06000002CC
:1056C000000100610111000E0D0778008601320112
:1056D0004902390242027C0E07800170004C0043EF
:1056E000004C00700080010B060000FF0111011149
:1056F000011101EE0B06FE00010101010101010192
:10570000820B06FF0101010101010182007C0C06F0
:105710000000FF0111011101110101010B06000040
:10572000FF01110011001100010C06FE0001010132
:105730000111019100F2010C06FF01100010001090
:10574000001000FF010804000000000000FF010736
:1057500004C00000010001FF0E070000FF01180057
:1057600024004200810000010C060000FF0100013E
:105770000001000100010E07FF010C003000C00015
:1057800030000C00FF010C06FF010600180020008D
:10579000C000FF010B06FE00010101010101010132
:1057A000FE0B06FF0111001100110011000E0C0686
:1057B000FE000101010141018101FE020C06FF0111
:1057C0001100110011002900C6010B0600008E0017
:1057D000110111011101E20B06000001000100FF9F
:1057E000010100010B06FF000001000100010001A2
:1057F000FF0D0703001C006000800160001C000317
:105800000D071F00600080017C00800160001F0EFA
:105810000783014400280010002800440083010D84
:1058200007030004000800F00108000400030E074D
:105830008101410121011101090105010301000755
:105840000008000A01001811101338313033787144
:105850007073C8C1C0C38881808384848782C5C4B3
:10586000C7C27574777235343732151417120207B0
:1058700002080201000301090304020402050305F2
:1058800000062024282C383C4044484C4669726D60
:10589000776172652025735F5632330D0A00252D1E
:1058A0003130732025732573000D0A5479706520FB
:1058B000273C636F6D6D616E643E203F2720666FED
:1058C0007220706172616D730D0A00557074696D9C
:1058D00065202575730D0A0025730D0A0D0A005603
:1058E0004F5941474552203E3E2000256300486500
:1058F0006C70004E6F20706172616D73004B657942
:10590000207072657373003C6B6579313E203C6B8F
:105910006579323E202E2E2E0044756D70206D6507
:105920006D6F7279004C6F6164206D656D6F727977
:1059300000637400436F6E736F6C652074696D65EE
:105940006F7574003C6D696E757465733E004765D4
:10595000742074696D6500747300536574207469F4
:105960006D65003C595959594D4D44443E203C48C1
:10597000484D4D53533E0074640055706461746526
:105980002074696D65003C6F66667365745F696E4F
:105990005F6D696E757465733E00546F67676C6503
:1059A00020646973706C6179206F757470757420F0
:1059B000746F20636F6E736F6C6500620052656177
:1059C00064206261747465727920766F6C746167AB
:1059D00065000000008001500080025000800350EC
:1059E000FC3F0150FC3F0250FC3F03502578000D66
:1059F0000A413A2000202025633A20000D0A533A3C
:105A000020000D0A4D3A20002020473A2025303250
:105A1000780D0A006661696C00253034692D2530E7
:105A200032692D2530326920253032693A253032ED
:105A3000693A2530326920257300253032783A25BD
:105A40003032783A253032692E25303269002530DF
:105A50003278203A202569202569203A20253032E5
:105A600078004E4F2052544300253032783A25308A
:105A700032783A2530327800253034782D2530328E
:105A8000782D2530327820202573004D4F4E00545C
:105A90005545005745440054485500465249005367
:105AA00041540053554E009DF070763335733DD010
:105AB0003C41E0E5DA6A4B89E179329F98755A9E5C
:105AC0001D4A800C326584961FE4C043E150DBE33D
:105AD0006B68244F74502D1C03540B30BBA9D8C5E0
:105AE00029AF70C9CBF28F3153829FC52F527458A2
:105AF000E010789976BB336B30F23823C065F243FF
:105B0000DAA098D09859FD5F61E9BA322867B933B5
:105B1000A8521D8A2E7C1AE734168F021473922124
:105B2000022463803C1057C93B81A453CC834B3083
:105B3000E3D9B54ECB994F66A4DF92C0377C10787D
:105B40007D02D050E88DAD55AAEF4B1748DD329C51
:105B50002E60996029C56F2FF7A16BB498572777EE
:105B60007E40E99C3809297E26E6C4A4CDB032DD0A
:105B7000EC049B8AAC69CE6D5B587537C847ABC3E4
:105B800006D05F490DF7D3728C03EE6C76DFD4003C
:105B900085DC6CC8D5FD314BBF1D386295A4BAFDBC
:105BA00012957BCC152ACCD4A8DF3B23F03FC063F1
:105BB0007CD76766C4035112DF568359C5C5E766B3
:105BC000F70C53D453E9DFAB48E4EA4EFC461FD14F
:105BD0004D19867BBC6F0D414F08058B53B8BB62D6
:105BE000807E36CB3C8CBB8B34022A5B837252D6D0
:105BF000A48FFB7C73C83776A23A827151C2274FBB
:105C0000E67FBB3A8BD720AD5ADBE778D301872DEF
:105C1000DA6CC57BA8873C5B168DD73C99BB9F8C03
:105C2000F5A4BFCBA22DCF3E36C6CB3CB66CC84147
:105C3000A93AFC1FC68E20D283DE0E67DC71F34AC0
:105C400036A26D24E1558C90C676296B70E9ED2162
:105C5000DF6463FFC8E42D7038876CFC4159595BE1
:105C6000084DCBD85EE3F04527E204E16D1CBEF49D
:105C7000C273E99F818CF866229A6D5D0744D02932
:105C8000BCD2CF6F549469E53AB6362D75DC116AF3
:105C9000EADE9814AA0AFF26502A63C3FD23E5967C
:105CA000320AEE5F9F98404CF4974EB591DE50510A
:105CB000F7A2FA2ECB81909D415DD9D8738F524BBC
:105CC000008B7658340886859CEE0F6385C6ADEE52
:105CD00038A60C32D822D9D2F69CAC47E96EA6C6BB
:105CE0001DBAFCBC8E6045B0AFC5E7D8214F5590BA
:105CF000F07798D6D734D300B99C7A8C51905C1148
:105D0000666BC60D6B2CAC8917F1058419F07BCC42
:105D10001F0E039A87DC289746F848F0FB22F6907E
:105D2000AB219DB31E7EF550CA1BF03ED59E30FFC1
:105D3000E1AF96CB027E43652248F9A8F9BAF95142
:105D40003B8100804C09365ACA4820B8C0DC4D72ED
:105D5000A4F7ACA54A4DED02DE7E4E9E8727BDC856
:105D6000F7A2658A4FB8D97E63125DF6FCCE99140E
:105D7000E3DE20C7F621DBD0296BEADBD6806D3B62
:105D8000B8328E4C35950B45D78E18F574AA55BD93
:105D90000B44307B6F1D91CF457611A21BC53AB2E3
:105DA0005EAD8C29294E379FD6BE3B7BF25D5A38BB
:105DB0004781097276829BF5831BD5740BBA0C352B
:105DC0008991186CE1CFC200D6CBCE84DCCEACB6C4
:105DD000379BFFA459D0F2EF973C9D230293FA879B
:105DE000E311C2594BFD55F776B590C9B2C7BBABAD
:105DF000784B9CCA4BE8592F21DCD3C937EC5F594B
:105E00005C5F1718F313073590C22BBC3C9A6D3CAE
:105E1000FF797CA2632A2D9AABA7A68FA670C3CF69
:105E20001AA90E7CADCF2934A9477C829975142C10
:105E3000063E88A93DF8F0BD47D88FCF48814A7902
:105E40003F42D30B3E4CD3376D49F1DCD59909481D
:105E5000B968264E6415F2FC99AC00563BFFA2A926
:105E60006B913564095A24042C528E32D47C1D0364
:105E700052188D4390FE62CFA7B43988A8BEC31FC5
:105E800097D675B21CACDF233EDAC44E690729D31E
:105E900007351D81A35A0202070477938FFDEAF8A4
:105EA000FB23D4E2BED524E9F17A6900AEA0D19CEF
:105EB000F25EF5C30D1C5E6B2D89E1EB43319AE96F
:105EC00097E41B4F8D1BD133B8DEFEE25A0C91A72D
:105ED00033C6BD44954182C69CB75EB1EEC04BCE81
:105EE000C37F6CA9334A5BFC93A9D0509DEB8E888D
:105EF000053577D6F34BF59755C4D79F20038EE42D
:105F0000245D77F41909E472C3CF09B17EA13D1372
:105F1000D8686A0375456FEFE1A90738B852B4A194
:105F200096006A8E8BE47803D5E2DC39170B3E903D
:105F300084B824B2A9F11D3957850288E654700D42
:105F4000E6FDED304FB623ADEE91DDAB43ED919123
:105F50009CBEF0595DBC267CA17653186D71F8FE8D
:105F6000D1A9E6C0BF72CFCE0127248A89F285F578
:105F70001373188CC83FE96A1F94FDC22689A3F9E0
:105F80008C10F5856EB6F2FD2274C3474EC9504D94
:105F900023E3562A83B9517C8E501D14854F93E319
:105FA0009F795132E363398D4B8F616AFB384EF72D
:105FB000B555A199EBCA969684D4230FEC72BEC650
:105FC00095E25DEE42F1BAC5711A857FADAD3391B0
:105FD00000E3545274507D4BD129ECD47DA0E01FD6
:105FE000208FAD183F7C721B165D806278050A8396
:105FF0006CA8753E9A2A045A80245FE8BFDC05012C
:1060000049892CDF022ADBCAC16B9706164EC7C628
:106010001E1E958EEC8987092D343A0056B5C6555B
:106020008F2B6407E00E6654B4851E4666B861EF98
:10603000E3AED971EE4A7DC57FC073B42394E5F712
:10604000CE6F42055F92FF4385FDC2917AD0F35334
:10605000E5A8306C15AB6F69C0C076676AB5623E63
:10606000D9F39AD8DD6C9ECBA30D36F0E2B54C6B1C
:10607000AD82658848444EE8A3740D22E26DE10FBD
:106080009474EA0CC17363E7F5D9309643930E3DDF
:10609000180A5D27624CD841AFD27408C0AA957126
:1060A000FB5A5AA467AEFA5E0004E6C9D12EE3A8F3
:1060B000EAA1C318A4B20F694A080E1294590DF54B
:1060C000EB49A2AB579FECA01697009A876ECC279E
:1060D000821872A4B3D045540A3B53EF6BB6EAE87A
:1060E000083E6E9C3C06B39C88657FC0B07B4087B1
:1060F000B68D4D200E15607FDC8138D2E58A85AFE4
:10610000C1A8EF2D0BAC92344346E97185179ABDB7
:10611000E8CA3CA78345161C97E3D3555A9A6039C1
:1061200092C1FBD4DF54E74660A62B485260D729C2
:10613000C660F9C6F11379C3EE87D99C03E0659078
:1061400088FDF1FBF23E1C28AC34F394D6B8CC4663
:106150005AB9EB212B75E1B45FDCC543EC8C7ED5DD
:1061600008EAB7E4CDAA83EC11765AA47AE783EB68
:10617000AAD291858A744DA232B1766CA21BEECC64
:106180000A446521B59D8164BADF3E0A5481260B1D
:10619000D2696CCF6A90577D3519B3C0B122B17501
:1061A000CC5F080C032A80CE0DA177F3B0990926A5
:1061B000324A955B9A8512483CA8B2DBF1CB498202
:1061C00028725EDB686B7265FB88EF3F4FD03951F8
:1061D000231142DE2D61334EED84A5B694D07C961A
:1061E000186B4674BA8BAD36AB2A98A2FB6F42B1DE
:1061F000F42D034AECB887768A08E20AD7ACDCD7DC
:106200005C1E847263813B7B985C1FD1032E2CF84B
:10621000E86344BA11A78C8A771128584A66C2905D
:10622000F30662F7391812C46DDBC94F515FB0979E
:106230005C4D378171CD52DC0E5FCD754953A07432
:10624000878504F4C3EFC881AD29E5D356E4E7237D
:106250006CA60676DFAFCF2771AFBA111982560F41
:106260009C9A76484DABA6B87BF7B4BD6A9FDB73AA
:10627000C5D4F9B3FF3DACCF226AE4DEB56CF89B20
:10628000E03251DBBEBEED80A3123110FE49A27395
:10629000E68BE8A5794D521909357E8A2C5AE51608
:1062A0005C5A2F20120BF0CABEA30918EA90CB9CAF
:1062B000FD666F9CD78E8ED60169A248012FAA6613
:1062C0009445391EC326C6F0FE240DEFDA60108B0C
:1062D0009FB70B989A9DA84FE131F45E1BBA37B473
:1062E000E10BB809FC5F53FAE63FE5FF62721D5C03
:1062F000ED71195D521AA7EEDA54F856FD915D441E
:106300004C9E3B0D59B572C71AE13E2A6D38B99AB9
:10631000417AFA63CBDCA36324F6FE0A36B9B001F6
:106320001E74D699F81085DD6778349156BC72B624
:10633000AED09B2AD79266656D58CC9EE27CCEBBD0
:106340009D05622B2AD11D40A61AEE77F06BF69BB5
:1063500015393E17F759965B7533B4DFAAFD872DC3
:10636000A7E8FE51605E0F6AF9FBD64C11FB4709A6
:10637000B4E67A54F5574D7A5930F70084957A7E11
:10638000D30D3B325C7BC98BF3EEF4BBBB0B029AA3
:106390001FA6DEC28F558F8632AE6584E3EFAE62F4
:1063A0006EFDD6A1E0AD0F8DA4075349D14238A0B0
:1063B000CCD322E7C41621508976133010BCFA865C
:1063C0001B2990FBF0EB4784A67DE0C7886A2A165C
:1063D000FB86D433C4BF6233974F1C401859010F5A
:1063E000F17C8EC6B15AB0915EB1575ACEE9194DC3
:1063F00098D6E2A985C9B5F89FE87FF05519893785
:10640000E6DD5815DE3CCEA1AC87160ED29A09E720
:10641000D4BB460BF0DC755CF5BCCBC727ECF6555E
:10642000FA035F10FDD7B5BFE327D1398304177195
:106430007FA78D363616152BC28B8D9E3B618EA1A4
:10644000946511281C662FE6BC6D71F8066712F77B
:106450004A4D3308AB4D111B54D747AA7E1A9941B8
:10646000F81C945CC995488D1B259F6B0A79F02315
:10647000582BD1A6E983BB0A07E4E5088DDDD2AE2F
:1064800063752D3D858BBAEF8E03CB14532EA0E997
:10649000EF834109BBA2432156E00AD00EE94D74B7
:1064A0008E454345913410EC348619B58563FFB8A9
:1064B000755CD67577FCE93B5726139A2CA85B30A0
:1064C00082B04EF933226A583C18EBE448CE6E6A2B
:1064D000414CD2FFEDDA0CE13B1DA814126424A557
:1064E00075F1B495FD129B3DCD9F3765C15FE5DC2D
:1064F0004CBF7F20D677FCC793A5EC7C6993DFD790
:106500005B07B584BE851BD860E2734F63117CFCCA
:10651000A9CCEE2DF665086F2985910C1106351C66
:1065200081A54813F4270C22902D149858448970A3
:106530003449B7C10138337046D4CECE38DFEFEDE1
:106540001E4DFAD7651E7B6A832078C998287B91F7
:1065500004FB0260A662692633298F08494D6D1C31
:1065600019031BB4607413BD134679AB9CFF8F8D68
:106570001B6D4EFF6FFC4B2EB089D848E12CB91231
:1065800061A1683982359F13201E93D05DAB11D66F
:106590009AFDAC0B69F4AC1E5D7E0D82E59D77EF34
:1065A000E51897B25C429CC8BEB83ABC22398A9DB5
:1065B000EB367C92F88208C1FDF23FD6104FACBAA0
:1065C000CEF509C8120C132E67AB9481FDD5C8B661
:1065D000449AE63F5B646B7CE7E0A0BB298E6E9437
:1065E00078C89A1D0C46410349C9B50F6D87BE8214
:1065F000DCE80DF07B68D2922ACA71BB9D003C6238
:106600000BB76C2D18E76003BF35BEBD3C17B8EE65
:106610004CE25BC3E476E948862CD3D8A0E8530863
:10662000F03AE7E966610DF374FFCAE2EB8BA69CD2
:10663000E6D4BDC89BB185B5D9A304B78EEACBD249
:10664000ABFCC32F60EAF18D2F1EA6205B7D436655
:10665000B1845C621673D39F3FE20180839F6EDA40
:106660008BC7E0D368AC266422B0606064BA0AE1EC
:106670008F003010E32F57038D7E9B79A3055C1AA2
:10668000E8B600C5EF06E0A073B57126EECF6C81C9
:1066900013E37E8D78FE64D26113FA860F29E83009
:1066A0001BF932FEF35262B56056340C784B8319F5
:1066B000282F6CB9FFC0FDE3D8FC83DA0E2A2666CA
:1066C000AA36F99D2E5429A9CC58434A8DFBED8654
:1066D000F40C7131504944B9B6C2593082F81BFFED
:1066E000D7E4135B6EB28E8CFD61F38B0ECF9C688A
:1066F000A8EB60850B65E77124E0B69BDDD86B786D
:1067000049D81F6296E840ED6027D008EC2ACA05F8
:1067100018DF6453FA08A1BA04760DC4CBA30FB3F3
:1067200080C39C2DC49AA6F47F0058FB1B00E95E31
:1067300089B6B41C270BFDC420367D622EAF2F8B8B
:106740005F96C72007863EFDD00B913D02D624D22E
:10675000840520FEDE6C355A0DAF6BC9CC2332BFE9
:1067600095099E77E799A515FE56041D81FFEDE674
:106770006E3171C57F73E7E1D4439722304D7C6D54
:10678000E4E290F5B01D414DBD061C0C5FD3B9305D
:10679000C9448DD05B1C392FD4A5D2DECA7CF93E0A
:1067A0005F7147D20BBE426EEB1CA887FB1FAE6425
:1067B000C863C554537F0ADA3E3C8780E66A5CAE04
:1067C000CE2E4394B18C8730DDFD3983239AAE7889
:1067D0008A6E45A07F8B3E5EDE6A747758610B6FD0
:1067E0007E02EA50D987069EDE73FA039DB89A6549
:1067F0000DEF616D59F97EADC4334ECA6CF2D2759E
:1068000001D58FF5830A63A28BC15B1798EBFC1E41
:106810007BF03738E9FF3901490CAFFA22049B1AA3
:106820009C8CE3334750274774B44CADFCE106958C
:10683000B2F5A48CD097FE6725739E2CC37A86BBD5
:10684000D159978143A9C9674AE467091ECEE9B8BF
:10685000D417EE2B36A98038A5A469B5D6E3E99103
:106860006D469A3BB740B2DF78A9E8C82C18702C67
:106870000DD47D045BAA263E39FAC354FDDB96167F
:10688000ADA016859EDC11BAFC96E5D82AD855C273
:1068900041FC7C0FE403371BBD6A09A1AD781FB32F
:1068A000C13B38903B4676DFD0147DA240B6B33C66
:1068B0008C468504D91F0AD23EBA3AAF3591513D74
:1068C0000EE6EEF74767F0A5E5214D216A9942AE45
:1068D00099BFAC75EE70618918763D32E173D6F7D9
:1068E0004BEE4EAABF3A5E3900887B645DFDA03254
:1068F00037C3FA08756944E12BE697F441E6FD5188
:106900009616E8349C4532F11E4D4DE3AD27FFADA0
:10691000671DF43A479EC70004AB98A5E485A3CC55
:10692000477EA45359BC5BB5A9F72E810B101B48B9
:1069300069C5051BAC690890E9F8C0FBA81AF76B9C
:10694000623CB508E1137981605CA7732D5557F05F
:1069500039F43011031C2416F02E870C61AEBB2EC7
:106960007B6029370FA161600709AFB356239BF7FE
:10697000B1C22D0F2764B3171C109D621CCC1829BF
:10698000B3D6C8640061667C37ADC16A9E979752E2
:10699000A888BCFA2DB2AA56130CE86072FE9F8F2D
:1069A0009CC9D0FEDA9171C02BDDDE94FE34838663
:1069B0006223717512782421406F9D2FB4B82FEE99
:1069C0006F78D5BA2E2E38756B7ADB9FCF33A6033E
:1069D0002D3BC5D02DD048931D4BE30DB6756E8968
:1069E00084E2382769D7C1C4B9CC9C830B541F8774
:1069F000B13A85B70D1AA979052B7A51F2F845837A
:106A00005016EC6991B446413DD8EDF2D95354EAA1
:106A1000A5AF24CB6291A6D0838997A1BD1A6BA59F
:106A20002890BC86596BAA1EE72B42DDB32F28B5F0
:106A3000A6FF57F0F7E8B5547948093D345F4F2A6F
:106A4000FF1C2196F62335DFF9C5714C951A0C0011
:106A500039E63CB8BF0F7EC2D9BD11ED45C3BC4D70
:106A60006C3BDD2C91D45D38D955B5EFC9EF1507D6
:106A7000E2702AA96D8A5DDB89E284D3AA5B8182F8
:106A8000295C03F977E0F0D5C3E040449BE0FA834A
:106A900067B6AB6599A9714AF14FEA5201B476D84D
:106AA0007C2732778F03B15DE9616FDA89BA795B50
:106AB000DE8770F14984BF33A39B31E0006794E027
:106AC000B9910C237AB9CF737ED7E0C2FAF5803042
:106AD000DB97C964AC4627EB3DBDB5BE1D577A1A9E
:106AE0002D82F091DDEDB569CF51FB13222950AF16
:106AF00074077C5C261871F3969B69F74CCF69A1EB
:106B00000D48B58B0831FD2C2AE65896D88E816D3C
:106B1000E61CAA75EED5E31C04B416BD37E13B585C
:106B2000775E6AA6552DB9744D874AD4DD50E612BA
:106B30008F46B9FD4970EB84963B39615EA2B3FC88
:106B4000AE84D15D1BDF0B6F1B5D6BAEE7F302976D
:106B500013204461F2FC25EB1C2E9CE0E810E08C35
:106B600067DA9CCB1D4729188122ED172BD65A34A2
:106B700060B9ABCBBAF117A966E7BFBB7EA6AA7B0B
:106B8000653CC9F7695EBEF9FA194463D0D9EFAA2A
:106B9000EC41AB7ED9F1F988BFF875851839430B04
:106BA000639D639FC53040C22A5927096E33821CFA
:106BB0000C72B73D4C7218FFA8C9D187D5DCEC46E2
:106BC000E6E12EB1E4513650A2332C4A02DCF0E467
:106BD000B1BEA93B7A27D467C4F6E124677C4BC8D1
:106BE00067E3D77920597482C8B70D4E5866C23D05
:106BF0006DDEB1F4AC0680234B1FDEA8A066B97D24
:106C000087184D8AF531B8B4FF18739A26F70C141B
:106C1000597E5E401B9B7987A0065753DFBD2946EE
:106C20006D97F0016D6BBF3F830F2FB6E951D4E62E
:106C3000CC69014579BE6B32A68BFFCD2085D5602E
:106C4000B5733AEC8A7084DF71B71BA99ECAE90953
:106C5000B91A9802146E2ADD5461F1DB85DE1E79C3
:106C6000C27E6FAF86B9B1ADDA61E4BEE2573B8157
:106C700073FDFA8143695147DFB4673BA55FFF515C
:106C800091044C7EBE6F4B01230A701DF3DDC1469B
:106C900010DBA7C20D68031720373A64BB1AB8028D
:106CA00058F72D74C1073A8D4A7A7E9AADA0DCF46C
:106CB000F953E880857CB9B508317A92FF555226A0
:106CC0005CEF875831239105C6486D8C67211058B9
:106CD00038130B2B187CC415DCC5837841B6A4BAD5
:106CE00026BE871AD986E0D43D3E98684FECCB6A21
:106CF000188E3D14B2B9A5EE03A1869F70C7D6A920
:106D0000AAA1B28AED706B46836EBC104F4A22B2C4
:106D10002A5C42B58DB7269D60E3EAA5A187FDA652
:106D20007B19CECAB518020F186CB46F49A2A6061B
:106D3000C2C455995FA3D3CAD46603039C911F5E56
:106D40000B74D3E83DFB64958531060C522BBE8D48
:106D50009A6D12BE17C654B59DB94331FCC364EF9A
:106D600093BB9F5CED373DD37C110945AC55DEDA12
:106D70008ABDA2807713D1A3C32051832F20A2E123
:106D80001463D6351E98F9D9293C0F13A874C10E87
:106D90006E27B573C59E4DB1CCA55A114819C9CC03
:106DA0006BD2F3790BF125A3BAA3EE6DDE6F92E3FC
:106DB0003D4E9D73E938E06ABC188C9D8758269A31
:106DC000C1252B214D9A72D14ABF0C1877E358EC9C
:106DD000FA6FFDB71D32A34F4179241C1F22B2E880
:106DE000AE4E84577FDE918D3B9B9E755974CEC409
:106DF000AB4CA96894BFF06384923BD1B1D3BFACD4
:106E0000AC66C1596D89DB3FDCC86BD513C1D90FA6
:106E1000D009A90E3144D09164D12A7DF41397573B
:106E200012B8F8C8BB79EE9521E9B5B127EE3DD788
:106E30008056388F163C5395AC8C0A4F123DAAC42D
:106E400015B1D309B30742D8CEFF9933B4B69A012E
:106E500031263CA95E0F09B3683F8E5E8D1CC718B2
:106E60009DED332676B1A3700F8ED8C35ABC32B4D1
:106E7000D7D1F9C60A6FEB1BFF2ABDB43764C5989A
:106E80004C830D5C4BCD5843C99C7BBB9C3CA7A558
:106E9000FA4F0CDE570F9C364A225F684A90F6DBA9
:106EA000E2DFFF238917873DC73FFA358759ED9DFC
:106EB00004A7B00FB3B9495B692DF031D1C80E36C4
:106EC000BFB606ED371472954F60543DB45EC830BE
:106ED0001382BF12DE8D039CC465499986222887E0
:106EE00075F8316F491899BD23ED48B6CB1539ECCB
:106EF0000B435DF006638A8579C9C1458835B0D1F9
:106F0000FBE79E3AB7C0DA8BF23D00B6C182AA3DDC
:106F10005D6F6679657A540BB39C2603DD8B25770C
:106F2000CB7EA8E8EBD61BB9C5FAB5B157CE65E55F
:106F30008433C8A4110BB6E92A79D0AE7FE70E6E70
:106F4000AB1A6A63F3D998EC27BC13EC0BDE1CB5C3
:106F5000D506B1B11BC4A004DCB2C5DD98311D5B00
:106F6000DB6217E9B4E00E5A4800AFD08CB6423B62
:106F70003682FCC8378F2D85A7B03BCDDBC94CFFCF
:106F8000FE159DDAE2AADEEB08A921FA517FDD7138
:106F9000890E895FBFED13D54EF80AC0C97F5E3AEE
:106FA000522DB38648907F04E2A694779FA51E20B9
:106FB000416EA4F7CDCA0DBD30CCBDB2727FF8CE04
:106FC0009BF5E651079D9734FD27D53DB9B0D5C156
:106FD00061B9A713A9C04A6E1ADC057681600E63F9
:106FE000598D5FDBC7D6EB958B52E57BDE7A564534
:106FF000BD8B8ED2164E456862B9462AA28F7E1D81
:10700000C845C334DDD7AAB8A7672BD9A8E1C1709A
:1070100083B2D0AED3A7510AA834E06610B00155B0
:10702000E7D1B53A204BFBB41E236B3FC00D695826
:10703000996B0186B2EE0BC7E537C6087C3F9859BD
:1070400077E5E7D667A09C08AB586C2EEFA96104E2
:107050009D78A2C157EEAE57F7B2B28DFC013FBF8B
:107060002084B2A4E3CC8ACF607F6ED79E999EBE67
:10707000106073E799DD4B114130A838EAA0872CE6
:1070800034718238CE046BDB26DEDC161FF28B51A6
:10709000693EDA444670C16A812725179C87D38DE3
:1070A00023D995E1CB945489C6393BC42000219A59
:1070B000AF658D329B3955F3ED281224531D4731AE
:1070C00028C361ECBC01884F4C76A7495517447C16
:1070D000E011904E95FAC526F6C1AAFD20D254F3D0
:1070E000E6461209F939B1377A19EF047BF7E4E380
:1070F000502815015B029B80E788870CD08FF9210F
:10710000D305AC24B04451310F055F5AB61DCE12E1
:1071100040354D2B531B5A5E113A184CF26D2926FF
:107120009E1CC305A52084BB7BDE659B5EA0023749
:10713000DBF213F7AA22E7103EAC2301D0CC5ADAD7
:10714000002F96B8BDF616EABA6824B7BE058ECAF7
:1071500011D41D273EF3630A9FE76D00DC5FD790D3
:107160008B342F9845C93A90F7CFF35A6A084FCD20
:10717000A7CC0050BC06496263D372CB76E426D319
:1071800008C4A9098305821FDA490999D523DE902D
:107190002D5DACE9194AAFC3F18B6BE780BFF62ACE
:1071A000D933E83802C69335609568B2A2EB044043
:1071B0008A467346466C4F482C8E6B2C42940F4C7B
:1071C0008753CAE32C6433E9247570B57139B2CCA6
:1071D000BF9708A4599E61BBF5F9A73B57B25D86DE
:1071E000DBA086E6197282D4868773F3A0B5DDCC66
:1071F000C9389E160FDCEF901CFBEF0179DF6FEBB7
:1072000091F59C36E8B9673E474EDF143B032B0FE0
:1072100092B8681E01BBC28EAA98D077DA519A1C28
:1072200091CC14418414BEBCD852B881D5B8A4A264
:1072300092FC036F3444519B0FC50AE41C9E532AF1
:10724000FB01BA30BD00FD9CDAC0B3E5FB9C737353
:10725000DD44E8F4CB7F7066C6D6E6ECD30A4C2654
:10726000DF212DBBF2DE689E8EBCCC3E0505600B97
:107270003DD1E6F73C7B1BAB15782723EEEB3C7E3C
:107280007ECB915FC17F396F89990D08695E246457
:107290008F2B72E178F4AACD457DCB4777F209D4E4
:1072A000C8532BC08BDA45FB57B40C6E125FE94C08
:1072B000118F78B779A65B3C19033CA815EBBBB0DE
:1072C00017636C1C99CEB11FED074353C5E3143E01
:1072D000026C368622DDD13BDEE7AFF9C78F0E2A7E
:1072E000395B5F18BF10B8CF114731A11A216D82E9
:1072F000A2ADFF7E2E32A178A78252939A2E7A9A5F
:1073000060555A2053F6C91172FE1EE72C3537829C
:10731000A5D2C03EB074A6304D09B1D24267311E2D
:107320000F706CEF4B5A155C477C6F825379A3FF4B
:10733000CD7FDECE63018A1131C3E580EB9E77C736
:107340001285CEDA5E9B5C7157565E07DEBDA7DA0A
:107350009B959B5E7C399960C18C20A79FF7BEE608
:10736000726579D822DB2063D76F28B5D05AD04810
:1073700082D70B090233D35A9E756490FBDD684DAA
:1073800093A927E51B47B69FA1C82B060F0F5D9C4D
:10739000BBBE8B1CB549880CA50F10A1A097FBC4E0
:1073A0004F0F573B39BB1BAF1352D9A12C687C48F8
:1073B000AAE937EFC6FC9BDC45F83AF47786FF1361
:1073C000D71B3B6784C7FD51839459F99764E6B096
:1073D00078CD1C57A17511846DC055867F7D3552BF
:1073E000F04088B26B660F3505E36167381C93C4C3
:1073F000081AD2471CE936C51D4CD0620D9C50DAE4
:107400006F50CEA623C93DEFD99D86A32EE64E0D23
:10741000AF34ACF92CEC277BE733A39DA9F1400FE7
:107420007F1AB0D0F5B0289F60B811447B5742A3B3
:107430009CBA515EAE2EC4D35FAB5BED4908DC5DF8
:107440008B5214BDE6ABF90C97E84C4ED5E8990F7A
:107450003245ED8EBC960C28FDEA618F4A0B23075E
:1074600025A43FF0ED7ED88CD140756A23B6D1F7C4
:10747000B69E2C67FBBF2F998F655DFF670FA5AB8D
:10748000EE6144677D51A758A1F4B48C445D2A187D
:10749000F82D1FCE69A026345746F92E99DBA74E4A
:1074A000C23ACF5031A2A3891A8B48957B6E85F3DF
:1074B000CE254021202DA4E0A5D3DA885957AFBBB3
:1074C000F48D7CB6586D4CBE3C12F0C1FC535797FE
:1074D000BA342A438042A24FD5A8980BBAC80C48A8
:1074E00081D6ED7CD171F5CCFD996F5E0BA8504132
:1074F000CED4E1923840BA5E7CF247DAECF039D86B
:10750000867946EB4F097571D90029813A6CF24EA4
:107510002A9EC1AB517C3F62655D7E8F5071E0F762
:107520000C5AEA93AA988610D0D5C358D3D3E2D286
:10753000042C671449C2C6ED5EC87B5B41A23D0BBB
:10754000234E0732F55C33E0CC95344A7EF4F47A6E
:10755000E664FAE6A2F19857BE96A13EEB1B5D9059
:10756000CBC8BFE13C1A168DA5F4B924F0D2C52CC6
:10757000A6B9A7EA8DA95E0231F438285BA818C124
:10758000BE278FFF9D98369BA77FC52A4AABDB2479
:10759000E467A1888C9C3CD6C7E6C1CB6DE515A9F4
:1075A000422E8E31CF2661018EAB420C1D905723A7
:1075B0004FBF3856B0C13DAE53FF2B76F245FC5657
:1075C0006C4C72D6217A2EB310C9A3F88A4C84165B
:1075D000C15025205DD6829368408998D9CE5972D2
:1075E0004F4074295FBCCA7A425CDE777C0A413D19
:1075F0009E123F88020F820D36B68C9E71D566F3BF
:107600009BBE43D98FE4BBD602F9B557CC449C6AE4
:10761000640E54D2B6E054A8B282322D733C793253
:10762000D3A386A87CC8C8ACFC023065DAB600617A
:107630008634A355B709A55B19C4FD0AAAEB9CA51E
:10764000FEAD35C3D0D4507F07C8D7B9B75F2C9FE4
:10765000F68DE1BC7548C1AFA69CCAEB9ECEC2F1C7
:10766000B51C0E8A51E9DCFBE64CBE2447F9261A0C
:1076700032877FBFCE2B3C856377A4C8E1886D56E7
:10768000CC986C48EE33B0DD740F01E0D133C2B159
:107690008F7E35B353E6A6715933DFA4F96FB087F7
:1076A00005BF6EF026B530D1F27ED4CC7759A41543
:1076B000CE27435697111E577A97C29A212F9EC5FF
:1076C0002680B07BE82ECAB439B55E6B3F04DE215C
:1076D000D9B5D9245FFE347A0C00DDFCD581C7B55D
:1076E000D8B6F6835B7402659B010BFC6BD38FAA43
:1076F000F81787EAF54370C723E68CEFD0810A902C
:10770000D13399FC43AE685242424BB618E61C0E88
:107710004D3724E14067ED55E0D64202EE6C53B997
:107720008E3D232439F8694275EBBD8A75C7D1C3F4
:107730008FE8E644C41793B994C66617C8AC757F42
:1077400081ADB3D86BEA7F39C9BE511529E487AB47
:107750001E9C398B86E460263A59530D04D1742659
:10776000371F8D17A3DBB5A50742962A2CA8D73162
:10777000D63D7F082B37700B96D780E6DCBB56D200
:10778000408B7995F638CAFE34DE15004EE426E9C2
:10779000ABD97FE75C48001AA3ECCC264DD98CE12D
:1077A0007C746CE93371BF7C8E44C5902A6715C820
:1077B000D61E57755565AB44B6A3D19E329FDD6387
:1077C0000FDC81C068A49DF1AF715618A6804640B9
:1077D0004DDD7B8B482C82588B7D683588F9F50907
:1077E00044D97127EDDEF19B1BD071F63471DF17A0
:1077F0009F5721253B580688E2C8C0108EB1C08132
:10780000E9A6356F2312CA22BB070F166DDCD372AF
:107810002201CD8412912986304D94089947E15B6D
:107820002D5177727D91264CF3AF3D9C3CD86BC8AF
:107830009DF98AAE11916F5954552498D49C965E47
:1078400037DE32275AE910BE6F4636A8AC47D273EE
:10785000964D0B82722CFBD83DAF918D5CB09BB5E1
:10786000EDAA2C63C296EF8B925656ED289C97F4A6
:10787000D447260D1BC6742AF3E0054550F35C7E01
:10788000E6FBE77782060FCD64CA9C922608CF49B3
:107890007A775D972575AC3409285278987B1469FE
:1078A000B86578C63190CA4370164D3F3FC28A759D
:1078B000C7DC1AF55E382280444951DB76BA4B307A
:1078C00024141B7A78000F7CF97F1EB9942ADEDC21
:1078D0007D8B7DB40D4E6BE7C9517E0F5156839A57
:1078E000D5B9CBEBF8D3A11B44EF69397681A10D53
:1078F0007C35839EB4A3465936B7130FA5A1D5D5C1
:10790000370630CF8D6BB4AEBAEB3E8BF3EE3FE370
:107910009A6CF62B3AA43CC954E4817D6652163722
:107920005F5B5D7C07189B1881BE0CDAB603A7AFBE
:107930009CBDD19C954DBC89DA527C5D27D764688B
:1079400079479D61039AE0F0BFE38CD63243C0AC27
:10795000FFEAE5E3923FA80097F02C22D70F13E44B
:107960009C0BA8B8C6FC0734D0E1760B256EB02E70
:107970008A286EACEC8267309BD49BFE2E406595C6
:107980002C426878F69E1C38EC487C31BC5591F24C
:10799000640056600A75FF29BE90C3FE7BD0BB7D94
:1079A000A41C44185CE7060E9A62EC507B6F087CBE
:1079B0003FC9FA7B0EF5A4BB6563C1EADBB0F59F56
:1079C000CB85C5DB971D83DEB83E0162F3CF501136
:1079D00023044BC9FBFB47FFAFEC00368D9AA25E38
:1079E0000708562501008A1A0337545E703F8D64DC
:1079F00097DE1E67B624769F3FEBB5E891A73E86DB
:107A00003A9144A7FD708193D2272F9AF65A36985F
:107A10008B99DF009CEE7289B4E19C3C52B76DB645
:107A20005F99345CE55F2A4BD450FD748165907A90
:107A3000C7E5976AC45C19F9E2AEC1FAFB9777749F
:107A4000904D7660E5EF9763C1C2805F5B0A812449
:107A500077B2D5E9544B253FBCC92AEACCBF140BF9
:107A600075B280C43D6EBC41A265CECF47D2F8FF4F
:107A70009B575AA066B5A25B0D11834A05752C91E0
:107A800083E64695A7D0C7478EB8C8D4491B5DD9B1
:107A90002D4E36E6A8EA52E8043884EE9AAD1AD4A0
:107AA0009CBBF40AA05FE0F1742FEA320C97CC8DF6
:107AB000BB1F392D6C5B37C5764C145A5307035DD9
:107AC00091E8BF69C33DD424A09D0E2F461771C213
:107AD0009109E5A92634B8708D2595F15E33A12969
:107AE0006AB2BA77B2CAA9572CB9364584ACF9261E
:107AF0003F8B12243FD24E80FB9737916F01B5E246
:107B0000B120BE3B384CC2362826BF59376098CECC
:107B1000E848F8683DB6B07543C2256F9044243AF2
:107B20007E80D16E45E1D4A8B65615E28C5AE4A702
:107B300019E331C004E19070402854F561BCFC5851
:107B400079782C4E9CE469BA505D2D438BE9EA713B
:107B50005CA5A8AF60E787D8374F6FB75E6A5A4D0C
:107B6000A1141894E56155118251888922D17D7B39
:107B7000484A53F9A8446258486568AD97A0BAE4EA
:107B80007003EC636CE8D7CF0F0396956408A4C329
:107B90000A71766BA2133B15D5A48AE53A004257C9
:107BA0002D41ECFAFC9B578013F592891968B25D60
:107BB000533FB0DD0EEE7F3E01840713CCC958F46D
:107BC000A39329E51CEEE252A02823BC84577080C1
:107BD0009E8290B9BEFA08B4F862B3FAD23625ACE8
:107BE000BEB2AACF382D97EA1A7D3D58FDB7A7DF60
:107BF000763B42DF2255E7F01160F8467131BD82D5
:107C00005C25274744EA849A8AAA3C8ABF72354990
:107C10001B4194B472A8DA1A90B24FE4B40006E69D
:107C200080F8F4B3B3057A3828655AF88CCD94EB14
:107C30008985511995B915D86FCEEC556306DFEAE1
:107C4000069A9F69CB2F1DE0C3E59805EC7260632F
:107C5000D426ABF568A95210459BA729B0F4E94397
:107C60005C5BD517E0B3BED1BAE5742D669BC787C0
:107C7000BF4BEEE31E3AF5F864891408F4F4053AB4
:107C8000732D34A59AFABE153DDEE05A4830F73F11
:107C90004F526738166BFEE60A01D8B7339E4E0A7C
:107CA000AE29EF3433A5CDD9E6CE77972741042A04
:107CB0009A8F3DB0F835C7D7F4DCA7BE6DF44EF807
:107CC0002A099CEBABC65A0EB4B0AEF2EECD3C42E4
:107CD0001F728F1A41E8FD762BD7FA7F6F7121E969
:107CE000D1F4186EF4C198FDBBCCFC2AA0560AEA68
:107CF0004519C904AC68B5889BA97148B85E02D023
:107D00005829A0FF0EEEAAA1F744C3827493A237AC
:107D100056B020B5BE42018E10A3D51C738BA1C3F3
:107D20005CE86DCACEEB15C9C78C7F2AEF6814C911
:107D30008F22EF6BBF45FED470F3ECA2888FD60F75
:107D4000D40B79E61E6BA49ACBB5B9FC6B19A134A0
:107D5000C619AABD400A6C13D39BB66BD5E7D47184
:107D6000797D50475C9B70C01B196313B02899B68E
:107D70003699EDB85844F90274A60DCA6405F1EEBF
:107D8000CDFA4AC0D42D38574AE24CF2C18C633543
:107D90005FB459F2D790A80274D86A712D4821A710
:107DA000CDF8849EC0994385467962EA611A0BE951
:107DB0007986D403AFD1C72EBCCA346CFF8842E9A0
:107DC00075EF2ED3EAD17B67A070506EDAE7B4EA84
:107DD000C4DCB0DCD3AA6ED7A3439012CD28EDF358
:107DE000B78C8B19118E90663A30D48AB69E54C7E0
:107DF000A89D4F1DAFAD6E131E0250BEA0750C00A6
:107E00007DFB75B19CA14B5F3F561F08D6C806C3CA
:107E10005888D6D248E6EF699E50CFF6E2D630F9C0
:107E2000CC1C77EFE478230303ABD40A724E26AB65
:107E3000AF9115B01A006AAE5C229A81BD2D9849A7
:107E40005445D5B6C7E8EE8A4E243215ED3F4DAB0A
:107E500052403B986B31ED09D83C00DD2CE9E357EB
:107E6000B94EB4A21DD9E0E16FAF2E4968EE2C8364
:107E70002436C6E3008E4E56786BA76FE19BAE6842
:107E8000F97215988A3F3D6061A78CF2D0825BC77A
:107E90002A94BEA0A0CB9958DB6C71A45C1763DA5E
:107EA00066A2591BCC8CBFF8CFFE696BAC5CEE4D63
:107EB000A125B96A36D0283704F9E51BCC5D906658
:107EC0005417081A210A5932BBB54307087051CA22
:107ED00096623598EDBEB799C566243AD6FF4D88AF
:107EE0006E3C78D958239B08F9842E3300B03DCEE0
:107EF000FB1C3F17579BD3F0A7EC194CF684409816
:107F000064D11DD8700CF4D534B5706C7452EF4F39
:107F10005B828DF2F6923EC4875BF19352988B910F
:107F200038DDC44359C315513CA9C34420A9336B60
:107F3000B1DBF15499F701B3FC49796FBB4C972B36
:107F4000FFD094A71CFEACA91756DAAED32A15862B
:107F5000BE0A3477285E38BEAA647CAF074E1EC2C4
:107F600026876BB597132118EFF91899C5B42E071A
:107F7000BE63713B58797BD6E3FDEE9E7BA4D209AC
:107F8000AC4DE3AD4A251F46A258344140F85CEDA4
:107F90009E7CFB7B21F2DF4AE886A56D8978ACF9EF
:107FA0000BA305BD9745E0999361E4130637D939D2
:107FB000F9F4B189FE250ACE406E82E496F1551C93
:107FC00032C21D4824DB4628C0BB3AD382CAB8055A
:107FD000B16ED00541771F19A94DEC1283739D93A3
:107FE000F191A77D2B6D6774A08926592559784397
:107FF000EA292491529CF057E06BABB06EE2F60E8A
:1080000004D51E60F35F4C0126DFC80DABD2D4F857
:1080100044611DD363A9E4AF0B47B29FFC7683771D
:108020001FAF58894D40995696C99448A555FCBF35
:10803000DE2107D719785B1241F5A8828DED09245E
:10804000B03C6C2C4BE7044F20ADB76F688B9706A4
:10805000835FA57AD6BA84BEBA6F7B62B5166039E3
:108060007992F6A82F5CCEFD2ACABE54F345BF16FE
:10807000E29CE4A4D3CF6BDFE56F886C77BB30C0A4
:10808000FD71AC1EB90F40FD20FA29EA457B9F091E
:1080900028198C66F4DB80D1DD657104B182FE6B3A
:1080A000262C446A3C68987A04F433C09221DCE2BE
:1080B000C232D0879ADD132E3DBCF324F39831B53C
:1080C000279A4A2123127BB411A3D7C7CA94E0266A
:1080D000B5E5B0086ECAADA97A4CA9A11C550A9D98
:1080E0001176E323B5F84E2043279CCCFA65F3D3F1
:1080F000980669C026960E7D9DC0E7BD73D1664A7D
:108100003BFB6F2A90C5C488BF079194732DF5334C
:108110005B51AB52AD40A5D848EA9553A357B7572A
:10812000559AC5A3A8A1CC970DDAB552ACDE8AF357
:10813000480BF2ACA7E758881E103D596B4FD65D2F
:10814000F73C9C4DB565C194B5379899328D6FA8B1
:10815000C5F9038A9ED07052F19EEA9BC80A23C2D9
:10816000601C791F905D7715A042F553546A064D47
:108170006C2400F8E1ECC9C38D0049F7F4E770C83E
:108180007AF35F2E28403CD2CE6C561C07573CA495
:10819000A2AE8CCF8D50F0E5DA5AF9B662EE72DC01
:1081A000C23753CCCBC5B726A115A0E94A3D53F33E
:1081B0005C5CF7E116CCCA9A01F4A1837DBB7CC755
:1081C000872DFE59F685D5208FD54E0717A8BD649B
:1081D0005958D30EBF48D843F7F7D3F50FDA26B571
:1081E0007EB197DC094611736FB7CD90AFE1A8124D
:1081F0008682A399319E7E3D2C398748BBB8EDAB72
:108200008A94E8057B59A30F4E5E516249272FE9F6
:10821000D4CE055BBD7024DE9BDB5811F23D849902
:10822000566CD753556879CCEB329255A872B5305D
:108230004872FF8D567250AA09E8C598555D90891D
:1082400072554F0F0BCC78B563C6E5547EB71D4908
:1082500059119D75616354A4FE46677A31C860F474
:10826000EB4BD9D32E14C5DFB14B53FFA7A520DFAD
:10827000C2D01F7874904BB73268E62E85F18DF826
:108280001063CF7E4776A05B69B421B857E8B3246A
:10829000ACBFDFB188E88E75AD99DE45D01967E0D7
:1082A000CA069D6463887DB53C064F2800D39ECFE7
:1082B000653B77D09DE9E4FBD242C5A8A1333216D5
:1082C00056A311F16F4543152DD3188314DF958004
:1082D0009916649D1164EEAB10FC1450BB4E899E40
:1082E0009F785C5F658A8EB3FA3086A9E79FF0328B
:1082F0004532E87791AF437B6CBFC0068E16DDDA5E
:108300002F6062A91932126E8B3E6DCAC6C2C14B74
:108310009FEB04BCB94CE8F2A8BF38C84C85B16EDD
:108320003C4A19F6E37A974880AE6619C5B17B28B6
:10833000F9BF4A26DE10F276F375B1419D77AD03A1
:10834000C419CEBF55FE27AA21B7EED3973B48915B
:10835000D3E343FD59D45D73AEDCCC488637BEDA37
:10836000A504B2F1DF8269FFE22CBEA3166AE9A67A
:10837000285D62BE07027C86DB1CAD2E30BCB0E9F6
:108380005F0B56E07E219CC4D7800C17B59841DC6A
:108390008BBD0CEE8D0D1733DDDC4B98310BF5F9F1
:1083A000334D0B4156EB0140D29CDEC54AF1C90664
:1083B000AD8EE9E0178E22C7A78B698C6C9989D89E
:1083C000674D35B2852FEA4CABB60B79D870E8CF44
:1083D000C8B8D720667856ACBC89649CAF241966AF
:1083E0004BD3AA46FB05BA589D132BB833E6792C1C
:1083F0000685105F6C86C8FB0584329C1FF2BD7336
:10840000706B4A2E11D80C453A1F86F3CAFB6C924A
:10841000D3AEAFB4BE9DA0FA1F03192DCD8B7A80C9
:1084200020D952D58B8857C1BA9BB8587159DF955E
:10843000880BDAF82CC263E309769D9DE1153F7441
:108440006315BEEEC540080F7DEB52AA9EB057C71C
:10845000D3E72E01B10D3AE6749F83BE623A5F9373
:10846000EDD4D6303C2F119A99D1FE0BD269301B36
:108470009880698D8FF8A5D439002B831C67C03D87
:1084800096AE9BED7F9A8E6AB51C374997B23775C9
:108490009C2AC19D0D276C77669686FECF22A0A5EB
:1084A0007ABAAD22402D0F9CA60701A9B6A19A8BDE
:1084B000523EA08CAFAD5EFEAB81F2AC4BA8889A69
:1084C000C2EBACCBFC9F2420EFBC23D516FDDBC751
:1084D00007715BFCE991FF46092121C4A6D704A6D8
:1084E0009E78C52033D039187DDE8A85EA4C018E0E
:1084F000C2FDDB6EEDAF4E17266015AECD31E6D373
:10850000CC141E3D17BC5F89346EC29898F7AC6CD2
:108510005C45051EA159CF70007FD45F8184AF1BDD
:1085200045C4CFEFA51CDCFBBEBB4EB742A0055B2C
:1085300076333F2B63A698899740295D0FC38082CD
:1085400034078193A8E291E84C980DA7D9D72D87DD
:10855000A901F63F861F5E228D3CA169F95A3FF8BA
:10856000B40823405B0F28803A63D62BB20B665ABF
:1085700005904EC7FCD0817CD472112CDB74AB8685
:10858000F1C9A7AF412293954E2F99E02E2D13F0FC
:108590003526459014A5326C10A2346E2A8FB04552
:1085A00002FCAFB607AEDAAF984B436463C6703BCC
:1085B000686A9F67A817A775101D1F1F85FA981F67
:1085C0006DBC4F0C2057B33717A30F7FB9B8F1D349
:1085D000FEFB9EBA8EC9AC3D012121C6ABD3EC8413
:1085E000082FE76F8D0EBE3349CA6AF9109B4F0CF6
:1085F0004B6F9BE0826C99B3F9C89C9792A1FAB932
:108600005F4B29EE4D78010C7E7880C0E1092CFE8D
:108610005D01786347B6BA5C1551FF5D21B20A3639
:1086200022EFE7FBD05D48B3BFB5528B99331ECC28
:10863000B7728E3D06866264983E2F719BE08D373F
:10864000CE50CCDDD889FB51307D15CBE04DF5EB1C
:10865000E90D79C74E2C61A2DEE2C469A221E5B121
:10866000746088A91A4BA6282A8F40DA19B655DA01
:10867000948F0FC06336FA7E087B2E0D55912EAA7B
:108680000775F4B5F3D24A59DC39443D1DB49993CA
:108690003B4BB64503DCB85A7F9F50BB24E9A61676
:1086A000765A3C2586B8C51C0224FE2CF24AE12EDF
:1086B0002388041F8F689E8C08D4FF03F87B47C56E
:1086C000E0B12DC31B8A3F8C6C8E6F95F6F2253777
:1086D000726B380C6621B159C5234BC39FCA0DC0BC
:1086E000FD6394D6B15AD02B4934FF89E4F84BDCB2
:1086F0000148B66398AFEA2AB629F9CA7C258702F1
:108700006E5BB790FDCE627EF3314FE8811BD0BB2C
:108710007780E75828838243C1DC94289D3F0F412E
:108720001E1754B1B570A8D039219500A35880C741
:1087300049733B6D952B74A2E547ADAB9A2928CDC3
:1087400033B7D073CDADBAC47D80A7F69B55302B1F
:1087500020968CB6D4DADEC2F8DA959E09588FB32B
:10876000FC322410E2DD9B2560602F62E4737B0005
:1087700083B61C14D881F154939CD51BD9A2ED3239
:10878000B64B238CE5BE27ADDEA3E7C8919A4FEC2C
:10879000005F1B808E523947FB4C650205599604D9
:1087A000565E9FAE3FB4901BBDCED1D75B8EB70552
:1087B0007E0B966B6AD916818532E52528FFA429A0
:1087C0009DE124B4701BDA2689D9DB319BE87EFD5C
:1087D0001069431A5B5136EC5878A14C729A2EBF3F
:1087E0007B2D982770610C4BDF5BEADCEE70A2AE4C
:1087F000F49D8D5C2ECBEFBB8C3B51752CD4898EB8
:10880000E40B6D612220FB85C0AE3AE7467A31C2A7
:108810006EF94C2529F0515A27F6392154E8836521
:1088200063444BFCF89F9FAD873D2BE745EB234B03
:10883000B4C057F88BC7897DFE33223C4D32CEBA87
:108840004A4B58009DF89111AC527820068A29F6BF
:108850002CA18864FCA837481EBCEABB9D6B1B8614
:10886000ABA47E12EE1262216EA3581B2CA63AD145
:10887000B79F18B9A7C8800808F1209E983E272204
:108880002A78D967A5666AAD18343A19E61EBFCEB4
:1088900068E7DB54B3F17FC297C7DBB585C78EC9E4
:1088A0007252AB6F6466664727BCB64514D4F41A9F
:1088B0006657067E018D5B534F9228E94AA4AAC0F1
:1088C000537C022DC0B9BCD929235FC54821C2857C
:1088D0004700E39AC3ECEF5E73B19746A7221428D2
:1088E0002BB158009EC835180A84050DD708B33738
:1088F0003C2399133BAB9C36BF5D2DC4CF18AAF91E
:10890000F72AC838CCF96DE90823CD84CF65BB3B85
:108910002FEF8D2C6B97D6EC0DA5FE92CC70FBC77C
:10892000E8D5D397529299F0768AB2CDC7FE07194F
:10893000124ECCC83A952DEA5AFBAD98BE96BD2290
:10894000ED5E72563AB311C374A837386A167DC209
:108950006498AFAAA0EBEE6F8D6C91DD28BD6075B9
:1089600057CE5D15F87790FA210DCA3B136368D393
:10897000FB80343A3315751827130A7C64F581C5DA
:10898000FEABF5DE6B8BFFA74ECBCF6DB85770B546
:10899000619CBD5D7287877C6B1068DBA6BCC08163
:1089A000E7AA8AC16EF8F16653E723BE0B26386545
:1089B0002CFB391501CB9565A399E6D24C03670CC6
:1089C000FDDAFA49EB6627090EDAD3F8198E42CCA4
:1089D000BEC9B1FF6122B90857341DDB238A72A1D9
:1089E000BE0824580A23132384FB7817EF8D4D49C2
:1089F00077C4E734E4384F4A0D1A810F68BC500B36
:108A000015EF404A00944B7BEBCB0AD457090C304E
:108A10007B5FFF7390ABDBA85F68D7FEECF6601856
:108A2000FF11E190D999B9CAB62040750E4AFE9659
:108A30001E100420B479BE2C13E547053FA873E34C
:108A400080D7BCD52905E9BFDA24A73C80212FA710
:108A50008134343A01AB812475C64D51333ACDA3EC
:108A6000CA96AE51460C16A32FED0F2AE230B70975
:108A7000EF3F284BC6C7921940BD60EA9FD7DA1D69
:108A8000A8662A17D6CE85700578E3AF796C6ECFCD
:108A90006987F6293A4E39E6DB7396A2F8977B4D43
:108AA000734A3510AB6B47074A421D58B1503EB66A
:108AB000F59DA1BF0A6D0DA7186477692873A336C9
:108AC0009F29329F7B5E085A0FA0B79037140A9DEA
:108AD0003419DD1F688B5AAEFF48F858BF55B4BD36
:108AE000736D42E79356A59DDA30BE80A08408FCE2
:108AF00023595B424A68C78AB7B4D8BFD15D274FB4
:108B0000D06CB42C4FBDE625DC69C41079F09A59BD
:108B1000B2843A389460645ACC1AB417BEC9B2DF32
:108B200097B35FE8540B2310B15EAB46A531AD1689
:108B3000170F9A59FE9AB8F5B73EE7ADDCB0F2834D
:108B4000401534700391B1F1D822D864BC1BBE0C1F
:108B500017286C608EE5956B4D49A4B36ECFDEFB94
:108B6000102E4E3D0AA03087E7FC26601CE5BE486B
:108B7000C426867262C2521CA172734B362DA95D47
:108B8000417F984E87BB7D1B71D1B53AFA27BF6DE7
:108B90000320405223FAE3055FB4350F222CA4953D
:108BA000E6CCF7C0B70D2D5AF245091E059B364D90
:108BB000AE5B0521181537C40E92B717CEE7BE1B62
:108BC0004FF16471055C6306DF1AFAE91A671367EF
:108BD0006C26988DFD245096BCC7050BB6D2136148
:108BE0005508390BB6C9175E377A73EF3F9732D005
:108BF000321DEBC78C70ED4E36193D0F38A40FA413
:108C00006FA296837C1EBE9980DCE9EDE5851B0191
:108C1000BF6E3157B8C910DE13288B9A80DEEBF592
:108C20009455123074F1BC75F08DA0BA3BE3380353
:108C300009EA052D55AF5E70A334F77C3750B2E1D9
:108C400002E8D4A9BF769907E4705BA6F3A5122CBD
:108C5000A2BEF4AC29691CF53882E40FFA4A03EC91
:108C60005C820036F2262A15CAD86A7D00EC06FD21
:108C700073FA9B1D5AD8FC4B2F463AE34953DBA6A7
:108C80004647155B0DABC43D8920478D7DEC329F77
:108C90001FD26B20118CB92629137E970F3D67D503
:108CA000BF9970FFB936CE3313FB094E0A35C87F22
:108CB00015A92DD976F8D61790AF81E0F0DD3041B7
:108CC0004F160149468EC7B92F48DF8BD78FA500B5
:108CD000DA937E2E34DB1F71183E417E602420A87B
:108CE000E54B2678CD53AE2DF31E019A591FD5D7EB
:108CF000A5B290C48D08FD492A939E7E40E4186B6E
:108D0000C8E20A188A0631F86C2276E93BF478FF4B
:108D10009684F88A8C66E3755949A79ACD18E27350
:108D20005624B6030B302445E87DDA8445730F2EB4
:108D30000B3ABA30DBEF3757F97F620F31A280521E
:108D4000651448988AA0EFA8A6219192AC8E30C5F0
:108D5000CC6C533D6E33D09C059B22336A2DED5570
:108D60001770FBF7142A109ED68FEE06125629E9CB
:108D70004CFB44F0FECABDE13D9D30B94CC838D72C
:108D8000FD2B361A8EC619153BA91E5378713A2849
:108D9000DE3DABE1374D960FC69C138AC37114DAE2
:108DA000A0C3A0FD8278312EA0667ACA195C613218
:108DB000BBCCE3C2D4575B4F7208744BA3019C2E0B
:108DC000172C0DF19D1E438665FBBD8F251F11A33A
:108DD000383D42A4195E14493727643583427E80AA
:108DE000B01A9613577D4ECAA2B917EB7BEBBE762D
:108DF000EC153122722EF78CBFB2A53E600BC0EA93
:108E000049C5BB8C6B869ED78E33B67BB6870DEC7F
:108E1000A8866538C6F312D05212FB6AD1B517374F
:108E2000FB1AE117930C968B6E22E95AC4FA2C2A8E
:108E3000FCB82D517DB19E4B1004818DFF95A73755
:108E4000FB402D4FB6B926DD2166246AE3E2201DE2
:108E500078AF87FFF82CA8E82BC0FD8BA15F05FC3D
:108E6000CEF03CA212CBCFC5E7C124E9BB09B9EAD9
:108E7000B8270DA786B5724E38B1008588FE478E9B
:108E8000FDCCFAB6AB0B7EA50438AACDCEF9357F62
:108E90008EF6096F7E323C27D4588A501304D609C7
:108EA000555A7B0C7B37CC6E021737B85A59C37EA4
:108EB0000004E8D6FB0D7F9C3CDFCB6B1B7818FED3
:108EC0002173859D3C352C79901B3E175115A5A02B
:108ED00056DAF73878207745702739136D2EB1A60A
:108EE0000695B955A21FA78B5AEF7ACFA22F7B41C7
:108EF00026A68D552DE8BD4445AF501777BCA8AFC9
:108F0000B205701D539F54B8D8815B9FEC3C4398C9
:108F1000A1FE9E1EF3624AC9B0B278A7F2BA0AFB5C
:108F2000D223B41C458E577B95F6B11FA81A0EBFED
:108F300005012D856A3BB6D7E55E3B89763A5B6EC7
:108F40000628204BFDC6448637D52802A7399489C8
:108F5000BF05EA9B9C18AB8FFC169EC00BA8EED4F5
:108F6000115F0DED3861D839A7253F6B600AD9A88C
:108F70006E87AAC8476E637738AE91F9DD1F3DFA58
:108F80003721258D9265B704371967A1E3A571B81C
:108F900049ED6B754AF82A5A4F69375CEC5C64F10D
:108FA0003F1DAB9802DE197C97DB53B004448CBDA7
:108FB000E13AD2B906D9543EB351856B6A3ED9E63F
:108FC000901D186A362DF56281644B9A546C961781
:108FD000B8B7F3AC3612EA4F2C27F2D6F3958E9A37
:108FE00061FCE78877B779D138B982F49B328B83FB
:108FF000262AD3DE87EF3F4CC84029D778EDDBE641
:109000002EC2870E618968F976D316293B5AC92387
:10901000DF40CEEE65AA15316AE91811F1F106A517
:109020009F31CD9D2CA2F2C2706E2DC6D0AFF389B8
:109030007C2E0FEE049B81AE8FE3B3DCD21AE248A4
:10904000FD4A71C9C64D05ACD89A99A423320105D1
:10905000BB966DB94FAEE9396FD83E11377441CA2E
:109060007329665E52F3059361F97B41703CF07B96
:1090700088BDC6BA45AEE260AE2E30D5476BFFEA7A
:109080001CA842EE20609CFFEEE2D7B04A1C7C8E0A
:10909000691F64C9E5945360E2FE61647A84CA3949
:1090A00041E27FCA8D4F7021250A5D103F7C56EE4C
:1090B0008272D4892594659187B69E865714F4A14F
:1090C000C3E784E485B731A1CDD0AA52274A7D6891
:1090D000D79DA67E762761F008BAC07BD660F9BF1F
:1090E0003B39C31E3FA6BBA0C3B7BB05CA58A08669
:1090F00046F5D96B9FFF5E9DA9F5055751E887AFEF
:109100002B07CE51B6160932F6D88EEEB16E44A7B3
:109110008483DB571DF3584F26B24C5E194BAAB11E
:1091200071588EA7AC153B78C4321BD7E15DB831BE
:1091300075BFD99DE77E382237D9DB556A90834EBB
:109140002D88F2CBB6D73A5F4FBBB0A42362D33A97
:1091500080A8CF61B5C2339254BD6B015AD9A0C16A
:109160003F4CB2EA53AE8C1D33A72F70135DA5227E
:1091700032DFFCF4F56CEA794C76A1EC25030F2D77
:109180005BEC6FFE97E5F409651BCB4F1F16D03CD7
:1091900079E09D622070B557EA1F02FD35AFD7BC5C
:1091A00035C82F2F30304450EC329F17E693898D0D
:1091B0001A683C73AC659AF97F47E4A592BA7518B2
:1091C000ADC009BED325565FF8D1F7E2C138737A36
:1091D000E7606E9F80757B2C50A308CAE24033BFC6
:1091E0005FD85AFB1D9F5454DBA6EF882F2D6FFECE
:1091F0003723DD40FAE066EAFC6C89B08AE6CFE30B
:109200003E939E11DC1DC57F24F7031DAC4422D77D
:10921000A07653F2EB8DC13F3272563F16AAE34857
:1092200033265289A55F0BC1B6968D4DF644CA24EC
:10923000FB746C011C7B8653D1C9E60F5778EF068F
:109240000E2EBA27A9AED2C2252B75DD1F8AD4A255
:10925000B361CA664C24DEBEB50A0503F85E3F67FB
:10926000232CC83DE4D06AC314B53D760DEE0B9AAD
:10927000F0DC782CF4ABDD75BA09715415DFCAA4A3
:109280003605DD435A3CB8BA5AB7AC1D28F3C01DA9
:109290000E05F7B2301D1EDF710D8868658294E4FB
:1092A000B3E59896FA8E1ECA5D98EC6E017E7057F3
:1092B0008ADFFAF7DFD4D35A5504047B0A9E2E6462
:1092C0000BEF1DEBF6B8814B04676716AD1AD4EEB1
:1092D0009753CB04DF8325B1B4AA42A95CCDA1E2A8
:1092E00058C35C3648878ADDEF320F4C3A491D1966
:1092F00093D524F64FED0D0526C42F864153E5D2B4
:10930000DD58EF26B5290741ABD0D37D3381FA87ED
:1093100083C89CA092953AB31E45C3FA79BEC0A3F8
:10932000EA02992709CFF653D3966CCC40FFF16A35
:10933000D79C9BE99CCD1F06B467F9B51BA7953C4C
:10934000C142C56605307086D2E7D2C238F0775A7E
:10935000617116B10B8A6B831BBEB947B19BE26288
:1093600008AD9557C7C986CCDDE446554C5E4640EE
:109370007A3D55EB3918264FDCFDC902D80AB132C7
:109380000EF811EFE86C65833202B9EE58F69CC313
:10939000409FA4F9BAA4C8E3F002EEAF98523D3A58
:1093A0008241D419286DB9AC2FA3472F7461E764AB
:1093B000E148407F7CF269974CFF1F7141D975737A
:1093C00046FA6A08326ADDFE0313DD4D1938B967C3
:1093D00072E30F090B6B3A8A8DDB970A58C68EE54C
:1093E00038A19E0738B19D8BE3C8F6802A8FA5A6C9
:1093F000ABB14EBFA7DEC3E1683F322A5C915D6925
:10940000DA5531737F8BFA28781BD2C66EFE75BF92
:10941000327CE5C5F4EE6767ADF2558304F4C78985
:1094200062533A1F18BF1B09E5C14400CBB3BA0E03
:1094300063CB7925DAF12ED9E701B5DF3672BCB0FE
:109440008D1B89A2891F283C056646A13ACB48930B
:10945000D17CA56810F4599AFDE90BAC4AC79F5816
:10946000465E826139C3DFF213C3CA5F3C431857BB
:1094700058AA9C8130F858BE15014810ED9EFA603C
:10948000DFCFF4332FA6A4F9BB30A9B1FAB69E5FA3
:10949000855CB92BDDE2465358ECD191496C845977
:1094A0000A1443C8B1C5C2D452AFCE3C275FCE2AFE
:1094B000BCE9AC117C2E937B25C7658BAFA7D38904
:1094C0002AE42B00301A58D52ED6BBB4B2B3F8C656
:1094D000E221936BA6809C57AD35D0695F84B9C1FA
:1094E000EA58BBF22FF6E88D6913CAA559735C8D53
:1094F000FDE877B3DBB77DEE610642BCDCF0DC4F04
:10950000A3C4ECA8A5D09DD76568A15E0D63D4D196
:10951000DF3F474CE512CBF72FCDF7B9D7255BE4FA
:109520001990C0CD82EB40A82130F67DA8F0285DCF
:10953000E4FC0422C35F3E080AB4A1260458F8E301
:1095400039494C57D37486C48884CE78F41AA5B3AD
:10955000B6F97CFF09D631649EA79BA183FC15FF59
:109560003F877572E006EDDA7A52DE105E1788EDFD
:1095700079D50B9289EBA5CBFECFFE7AAFEED0BDAD
:10958000DE6AD9FBE609F00F9070F2954C729E638B
:10959000761698B656E1F944DA5C845BAF266CDA4D
:1095A00057F00C6585AB08CF75B2A47A6EDC409994
:1095B00057FD089713BEB23B1825680BAF19759578
:1095C000B7F99DF4C74AA35E3C581CE2EAA197A4F0
:1095D0003D4C00750D99AA7362DA9D2AB53274C1AB
:1095E0000E3D43589B1C19FD867974CE92FDD9A07F
:1095F0000EEA5A6A98AA0FFCB10B6D0A78F414D2DD
:10960000C445C4169ADE6F9E6300326839BCCEE64C
:109610002654BD903058C0D948FB159F33E6CE0084
:10962000FEA8FEB78A309D3A7A013FB016F6FCF7E5
:109630005D080519128CD03CB24CC41A44D61F5F89
:109640007829BFDB3CCD2194C9C7F114E06E3B0EF5
:109650005399669DAE175E5BE8EB79C4D73AE1613A
:109660007F613A709D746268B60BE70CF9386A93B3
:109670009AB513E6B169BEE60981902C7CB2AE477B
:10968000F5C94DC1B2288C882C2FA71C743079D90C
:109690009EC843101CB8A9DBCEA139EC37EB4A6A4F
:1096A000837732FF0024AF0304050A08060BFF028C
:1096B00009070D010C00FF20256920256920256977
:1096C0002D256900202025633A25690020202020CF
:1096D0005F5F7C002C00610044697370206F6666D8
:1096E0000D0A005553455200460047004245474980
:1096F0004E0052414400442E4D59005052474D00F7
:10970000555345522020200066202000672020006D
:10971000424547494E20202020200052414420202D
:109720002000442E4D592020200043202020000DF1
:109730000C205A5F5100000D0C205A5A55000005AC
:109740000000000307206199500000FFFFFFFF4D5C
:10975000000000694F000000000000D11B0000EE77
:10976000580000F3580000F1580000FF000000A16D
:10977000100000FD58000007590000895A00000041
:10978000000000C90E000019590000F3580000172E
:109790005A000000000000690F000025590000F386
:1097A000580000315900000100000025110000346C
:1097B000590000445900003259000000000000F137
:1097C0000D00004E590000F35800005759000002E8
:1097D000000000510E00005A590000635900007744
:1097E00059000001000000910E00007A5900008627
:1097F0005900007859000000000000F91000009A9C
:10980000590000F3580000BB59000000000000DDC3
:109810000D0000BD590000F35800008B5A00008F66
:109820005A0000935A0000975A00009B5A00009F6C
:109830005A0000A35A0000DE580000FFFFFFFF0F90
:10984000000000F401000004010301020101041101
:10985000040F041704160118010000009700000807
:109860009700000C97000010970000EA9600001B7C
:10987000970000229700002A970000FB960000083E
:109880001C242C4448586C740502050804080B0875
:109890000404050105040908090406080702060274
:1098A0000402060106040701030803040C080D0264
:1098B0000C0203020C010C040D010D080D0408023A
:1098C0000808070802020704080108040902090140
:1098D0000A080B020A0201080A010A040B01020825
:1098E00002041008110210021108100110041101E5
:1098F000120212011302130812080F0812041301B6
:10990000130414021401150215081408170814048E
:10991000150115041702170119081A021902160277
:10992000190119041A01160816041B021B081A084B
:1099300018021A041B011B04180818040B04202029
:10994000202020202020202000000001000000E333
:10995000960000E8960000EA960000EC960000EA07
:10996000960000F2960000F6960000675A0000FB91
:039970009600005E
:00000001FF
